 windowsaccessbridge-32

 Timestamp is ffffffff (Sun Feb  7 06:28:15 2106)

 Preferred load address is 10000000

 Start         Length     Name                   Class
 0001:00000000 00006c79H .text$mn                CODE
 0002:00000000 00000108H .idata$5                DATA
 0002:00000108 00000004H .00cfg                  DATA
 0002:0000010c 00000004H .CRT$XCA                DATA
 0002:00000110 00000004H .CRT$XCZ                DATA
 0002:00000114 00000004H .CRT$XIA                DATA
 0002:00000118 00000004H .CRT$XIZ                DATA
 0002:0000011c 00000004H .CRT$XPA                DATA
 0002:00000120 00000004H .CRT$XPZ                DATA
 0002:00000124 00000004H .CRT$XTA                DATA
 0002:00000128 00000008H .CRT$XTZ                DATA
 0002:0000012c 00000000H .gfids$y                DATA
 0002:00000130 000034c8H .rdata                  DATA
 0002:000035f8 0000012cH .rdata$r                DATA
 0002:00003724 00000004H .rdata$sxdata           DATA
 0002:00003728 000002b8H .rdata$zzzdbg           DATA
 0002:000039e0 00000004H .rtc$IAA                DATA
 0002:000039e4 00000004H .rtc$IZZ                DATA
 0002:000039e8 00000004H .rtc$TAA                DATA
 0002:000039ec 00000004H .rtc$TZZ                DATA
 0002:000039f0 00000120H .xdata$x                DATA
 0002:00003b10 00000e44H .edata                  DATA
 0002:00004954 000000a0H .idata$2                DATA
 0002:000049f4 00000014H .idata$3                DATA
 0002:00004a08 00000108H .idata$4                DATA
 0002:00004b10 0000051cH .idata$6                DATA
 0003:00000000 00000028H .data                   DATA
 0003:00000028 00000078H .data$r                 DATA
 0003:000000a0 000003a4H .bss                    DATA
 0004:00000000 00000120H .rsrc$01                DATA
 0004:00000120 00000648H .rsrc$02                DATA

  Address         Publics by Value              Rva+Base       Lib:Object

 0000:00000000       ___guard_iat_table         00000000     <absolute>
 0000:00000000       ___AbsoluteZero            00000000     <absolute>
 0000:00000000       ___hybrid_code_map_count   00000000     <absolute>
 0000:00000000       ___guard_longjmp_table     00000000     <absolute>
 0000:00000000       ___guard_fids_count        00000000     <absolute>
 0000:00000000       ___x64_code_ranges_to_entry_points 00000000     <absolute>
 0000:00000000       ___guard_eh_cont_count     00000000     <absolute>
 0000:00000000       ___hybrid_code_map         00000000     <absolute>
 0000:00000000       ___enclave_config          00000000     <absolute>
 0000:00000000       ___arm64x_redirection_metadata_count 00000000     <absolute>
 0000:00000000       ___arm64x_redirection_metadata 00000000     <absolute>
 0000:00000000       ___hybrid_auxiliary_iat    00000000     <absolute>
 0000:00000000       ___arm64x_extra_rfe_table_size 00000000     <absolute>
 0000:00000000       ___arm64x_extra_rfe_table  00000000     <absolute>
 0000:00000000       ___x64_code_ranges_to_entry_points_count 00000000     <absolute>
 0000:00000000       ___guard_iat_count         00000000     <absolute>
 0000:00000000       ___guard_eh_cont_table     00000000     <absolute>
 0000:00000000       ___arm64x_native_entrypoint 00000000     <absolute>
 0000:00000000       ___dynamic_value_reloc_table 00000000     <absolute>
 0000:00000000       ___guard_longjmp_count     00000000     <absolute>
 0000:00000000       ___volatile_metadata       00000000     <absolute>
 0000:00000000       ___guard_fids_table        00000000     <absolute>
 0000:00000001       ___safe_se_handler_count   00000001     <absolute>
 0000:00000100       ___guard_flags             00000100     <absolute>
 0000:00000000       ___ImageBase               10000000     <linker-defined>
 0001:00000000       _PrintDebugString          10001000 f   AccessBridgeDebug.obj
 0001:0000004a       ___local_stdio_printf_options 1000104a f i AccessBridgeDebug.obj
 0001:00000050       __vfprintf_l               10001050 f i AccessBridgeDebug.obj
 0001:00000074       _finalizeFileLogger        10001074 f   AccessBridgeDebug.obj
 0001:0000008d       _fprintf                   1000108d f i AccessBridgeDebug.obj
 0001:000000a5       _getTimeStamp              100010a5 f   AccessBridgeDebug.obj
 0001:000000d3       _initializeFileLogger      100010d3 f   AccessBridgeDebug.obj
 0001:00000195       _printf                    10001195 f i AccessBridgeDebug.obj
 0001:000001b3       ??0AccessBridgeEventHandler@@QAE@XZ 100011b3 f   AccessBridgeEventHandler.obj
 0001:0000020e       ??1AccessBridgeEventHandler@@QAE@XZ 1000120e f   AccessBridgeEventHandler.obj
 0001:0000020e       @_guard_check_icall_nop@4  1000120e f   MSVCRT:guard_support.obj
 0001:0000020e       ??1AccessBridgeMessageQueue@@QAE@XZ 1000120e f   AccessBridgeMessageQueue.obj
 0001:00000211       ?fireCaretUpdate@AccessBridgeEventHandler@@QAEXJ_J0@Z 10001211 f   AccessBridgeEventHandler.obj
 0001:00000233       ?fireFocusGained@AccessBridgeEventHandler@@QAEXJ_J0@Z 10001233 f   AccessBridgeEventHandler.obj
 0001:00000255       ?fireFocusLost@AccessBridgeEventHandler@@QAEXJ_J0@Z 10001255 f   AccessBridgeEventHandler.obj
 0001:00000277       ?fireJavaShutdown@AccessBridgeEventHandler@@QAEXJ@Z 10001277 f   AccessBridgeEventHandler.obj
 0001:00000288       ?fireMenuCanceled@AccessBridgeEventHandler@@QAEXJ_J0@Z 10001288 f   AccessBridgeEventHandler.obj
 0001:000002aa       ?fireMenuDeselected@AccessBridgeEventHandler@@QAEXJ_J0@Z 100012aa f   AccessBridgeEventHandler.obj
 0001:000002cc       ?fireMenuSelected@AccessBridgeEventHandler@@QAEXJ_J0@Z 100012cc f   AccessBridgeEventHandler.obj
 0001:000002ee       ?fireMouseClicked@AccessBridgeEventHandler@@QAEXJ_J0@Z 100012ee f   AccessBridgeEventHandler.obj
 0001:00000310       ?fireMouseEntered@AccessBridgeEventHandler@@QAEXJ_J0@Z 10001310 f   AccessBridgeEventHandler.obj
 0001:00000332       ?fireMouseExited@AccessBridgeEventHandler@@QAEXJ_J0@Z 10001332 f   AccessBridgeEventHandler.obj
 0001:00000354       ?fireMousePressed@AccessBridgeEventHandler@@QAEXJ_J0@Z 10001354 f   AccessBridgeEventHandler.obj
 0001:00000376       ?fireMouseReleased@AccessBridgeEventHandler@@QAEXJ_J0@Z 10001376 f   AccessBridgeEventHandler.obj
 0001:00000398       ?firePopupMenuCanceled@AccessBridgeEventHandler@@QAEXJ_J0@Z 10001398 f   AccessBridgeEventHandler.obj
 0001:000003ba       ?firePopupMenuWillBecomeInvisible@AccessBridgeEventHandler@@QAEXJ_J0@Z 100013ba f   AccessBridgeEventHandler.obj
 0001:000003dc       ?firePopupMenuWillBecomeVisible@AccessBridgeEventHandler@@QAEXJ_J0@Z 100013dc f   AccessBridgeEventHandler.obj
 0001:000003fe       ?firePropertyActiveDescendentChange@AccessBridgeEventHandler@@QAEXJ_J000@Z 100013fe f   AccessBridgeEventHandler.obj
 0001:0000042c       ?firePropertyCaretChange@AccessBridgeEventHandler@@QAEXJ_J0HH@Z 1000142c f   AccessBridgeEventHandler.obj
 0001:00000454       ?firePropertyChildChange@AccessBridgeEventHandler@@QAEXJ_J000@Z 10001454 f   AccessBridgeEventHandler.obj
 0001:00000482       ?firePropertyDescriptionChange@AccessBridgeEventHandler@@QAEXJ_J0PAG1@Z 10001482 f   AccessBridgeEventHandler.obj
 0001:000004aa       ?firePropertyNameChange@AccessBridgeEventHandler@@QAEXJ_J0PAG1@Z 100014aa f   AccessBridgeEventHandler.obj
 0001:000004d2       ?firePropertySelectionChange@AccessBridgeEventHandler@@QAEXJ_J0@Z 100014d2 f   AccessBridgeEventHandler.obj
 0001:000004f4       ?firePropertyStateChange@AccessBridgeEventHandler@@QAEXJ_J0PAG1@Z 100014f4 f   AccessBridgeEventHandler.obj
 0001:0000051c       ?firePropertyTableModelChange@AccessBridgeEventHandler@@QAEXJ_J0PAG1@Z 1000151c f   AccessBridgeEventHandler.obj
 0001:00000544       ?firePropertyTextChange@AccessBridgeEventHandler@@QAEXJ_J0@Z 10001544 f   AccessBridgeEventHandler.obj
 0001:00000566       ?firePropertyValueChange@AccessBridgeEventHandler@@QAEXJ_J0PAG1@Z 10001566 f   AccessBridgeEventHandler.obj
 0001:0000058e       ?firePropertyVisibleDataChange@AccessBridgeEventHandler@@QAEXJ_J0@Z 1000158e f   AccessBridgeEventHandler.obj
 0001:000005b0       ?setCaretUpdateFP@AccessBridgeEventHandler@@QAEXP6AXJ_J0@ZPAVWinAccessBridge@@@Z 100015b0 f   AccessBridgeEventHandler.obj
 0001:000005e2       ?setFocusGainedFP@AccessBridgeEventHandler@@QAEXP6AXJ_J0@ZPAVWinAccessBridge@@@Z 100015e2 f   AccessBridgeEventHandler.obj
 0001:00000614       ?setFocusLostFP@AccessBridgeEventHandler@@QAEXP6AXJ_J0@ZPAVWinAccessBridge@@@Z 10001614 f   AccessBridgeEventHandler.obj
 0001:00000646       ?setJavaShutdownFP@AccessBridgeEventHandler@@QAEXP6AXJ@ZPAVWinAccessBridge@@@Z 10001646 f   AccessBridgeEventHandler.obj
 0001:00000683       ?setMenuCanceledFP@AccessBridgeEventHandler@@QAEXP6AXJ_J0@ZPAVWinAccessBridge@@@Z 10001683 f   AccessBridgeEventHandler.obj
 0001:000006c0       ?setMenuDeselectedFP@AccessBridgeEventHandler@@QAEXP6AXJ_J0@ZPAVWinAccessBridge@@@Z 100016c0 f   AccessBridgeEventHandler.obj
 0001:000006fd       ?setMenuSelectedFP@AccessBridgeEventHandler@@QAEXP6AXJ_J0@ZPAVWinAccessBridge@@@Z 100016fd f   AccessBridgeEventHandler.obj
 0001:0000073a       ?setMouseClickedFP@AccessBridgeEventHandler@@QAEXP6AXJ_J0@ZPAVWinAccessBridge@@@Z 1000173a f   AccessBridgeEventHandler.obj
 0001:0000076c       ?setMouseEnteredFP@AccessBridgeEventHandler@@QAEXP6AXJ_J0@ZPAVWinAccessBridge@@@Z 1000176c f   AccessBridgeEventHandler.obj
 0001:0000079e       ?setMouseExitedFP@AccessBridgeEventHandler@@QAEXP6AXJ_J0@ZPAVWinAccessBridge@@@Z 1000179e f   AccessBridgeEventHandler.obj
 0001:000007d0       ?setMousePressedFP@AccessBridgeEventHandler@@QAEXP6AXJ_J0@ZPAVWinAccessBridge@@@Z 100017d0 f   AccessBridgeEventHandler.obj
 0001:0000080d       ?setMouseReleasedFP@AccessBridgeEventHandler@@QAEXP6AXJ_J0@ZPAVWinAccessBridge@@@Z 1000180d f   AccessBridgeEventHandler.obj
 0001:0000084a       ?setPopupMenuCanceledFP@AccessBridgeEventHandler@@QAEXP6AXJ_J0@ZPAVWinAccessBridge@@@Z 1000184a f   AccessBridgeEventHandler.obj
 0001:00000887       ?setPopupMenuWillBecomeInvisibleFP@AccessBridgeEventHandler@@QAEXP6AXJ_J0@ZPAVWinAccessBridge@@@Z 10001887 f   AccessBridgeEventHandler.obj
 0001:000008c4       ?setPopupMenuWillBecomeVisibleFP@AccessBridgeEventHandler@@QAEXP6AXJ_J0@ZPAVWinAccessBridge@@@Z 100018c4 f   AccessBridgeEventHandler.obj
 0001:00000901       ?setPropertyActiveDescendentChangeFP@AccessBridgeEventHandler@@QAEXP6AXJ_J000@ZPAVWinAccessBridge@@@Z 10001901 f   AccessBridgeEventHandler.obj
 0001:00000941       ?setPropertyCaretChangeFP@AccessBridgeEventHandler@@QAEXP6AXJ_J0HH@ZPAVWinAccessBridge@@@Z 10001941 f   AccessBridgeEventHandler.obj
 0001:00000976       ?setPropertyChangeFP@AccessBridgeEventHandler@@QAEXP6AXJ_J0PAG11@ZPAVWinAccessBridge@@@Z 10001976 f   AccessBridgeEventHandler.obj
 0001:000009a8       ?setPropertyChildChangeFP@AccessBridgeEventHandler@@QAEXP6AXJ_J000@ZPAVWinAccessBridge@@@Z 100019a8 f   AccessBridgeEventHandler.obj
 0001:000009e8       ?setPropertyDescriptionChangeFP@AccessBridgeEventHandler@@QAEXP6AXJ_J0PAG1@ZPAVWinAccessBridge@@@Z 100019e8 f   AccessBridgeEventHandler.obj
 0001:00000a1d       ?setPropertyNameChangeFP@AccessBridgeEventHandler@@QAEXP6AXJ_J0PAG1@ZPAVWinAccessBridge@@@Z 10001a1d f   AccessBridgeEventHandler.obj
 0001:00000a52       ?setPropertySelectionChangeFP@AccessBridgeEventHandler@@QAEXP6AXJ_J0@ZPAVWinAccessBridge@@@Z 10001a52 f   AccessBridgeEventHandler.obj
 0001:00000a87       ?setPropertyStateChangeFP@AccessBridgeEventHandler@@QAEXP6AXJ_J0PAG1@ZPAVWinAccessBridge@@@Z 10001a87 f   AccessBridgeEventHandler.obj
 0001:00000abc       ?setPropertyTableModelChangeFP@AccessBridgeEventHandler@@QAEXP6AXJ_J0PAG1@ZPAVWinAccessBridge@@@Z 10001abc f   AccessBridgeEventHandler.obj
 0001:00000afc       ?setPropertyTextChangeFP@AccessBridgeEventHandler@@QAEXP6AXJ_J0@ZPAVWinAccessBridge@@@Z 10001afc f   AccessBridgeEventHandler.obj
 0001:00000b31       ?setPropertyValueChangeFP@AccessBridgeEventHandler@@QAEXP6AXJ_J0PAG1@ZPAVWinAccessBridge@@@Z 10001b31 f   AccessBridgeEventHandler.obj
 0001:00000b66       ?setPropertyVisibleDataChangeFP@AccessBridgeEventHandler@@QAEXP6AXJ_J0@ZPAVWinAccessBridge@@@Z 10001b66 f   AccessBridgeEventHandler.obj
 0001:00000ba6       ??0AccessBridgeJavaVMInstance@@QAE@PAUHWND__@@0JPAV0@@Z 10001ba6 f   AccessBridgeJavaVMInstance.obj
 0001:00000bed       ??1AccessBridgeJavaVMInstance@@QAE@XZ 10001bed f   AccessBridgeJavaVMInstance.obj
 0001:00000c37       ?findABJavaVMInstanceFromJavaHWND@AccessBridgeJavaVMInstance@@QAEPAV1@PAUHWND__@@@Z 10001c37 f   AccessBridgeJavaVMInstance.obj
 0001:00000c73       ?findAccessBridgeWindow@AccessBridgeJavaVMInstance@@QAEPAUHWND__@@J@Z 10001c73 f   AccessBridgeJavaVMInstance.obj
 0001:00000cba       ?initiateIPC@AccessBridgeJavaVMInstance@@QAEJXZ 10001cba f   AccessBridgeJavaVMInstance.obj
 0001:00000d79       ?sendMemoryPackage@AccessBridgeJavaVMInstance@@QAEHPADJ@Z 10001d79 f   AccessBridgeJavaVMInstance.obj
 0001:00000e34       ?sendPackage@AccessBridgeJavaVMInstance@@QAEJPADJ@Z 10001e34 f   AccessBridgeJavaVMInstance.obj
 0001:00000e89       __vsnprintf_l              10001e89 f i AccessBridgeJavaVMInstance.obj
 0001:00000ebc       _sprintf                   10001ebc f i AccessBridgeJavaVMInstance.obj
 0001:00000ed6       ??0AccessBridgeMessageQueue@@QAE@XZ 10001ed6 f   AccessBridgeMessageQueue.obj
 0001:00000ee9       ??0AccessBridgeQueueElement@@QAE@PADH@Z 10001ee9 f   AccessBridgeMessageQueue.obj
 0001:00000f3b       ??0bad_alloc@std@@QAE@ABV01@@Z 10001f3b f i AccessBridgeMessageQueue.obj
 0001:00000f53       ??0bad_alloc@std@@QAE@XZ   10001f53 f i AccessBridgeMessageQueue.obj
 0001:00000f6b       ??0exception@std@@QAE@ABV01@@Z 10001f6b f i AccessBridgeMessageQueue.obj
 0001:00000f94       ??1AccessBridgeQueueElement@@QAE@XZ 10001f94 f   AccessBridgeMessageQueue.obj
 0001:00000f9e       ??1bad_array_new_length@std@@UAE@XZ 10001f9e f i MSVCRT:throw_bad_alloc.obj
 0001:00000f9e       ??1bad_alloc@std@@UAE@XZ   10001f9e f i AccessBridgeMessageQueue.obj
 0001:00000faf       ??_Eexception@std@@UAEPAXI@Z 10001faf f i AccessBridgeMessageQueue.obj
 0001:00000faf       ??_Gbad_alloc@std@@UAEPAXI@Z 10001faf f i AccessBridgeMessageQueue.obj
 0001:00000faf       ??_Gexception@std@@UAEPAXI@Z 10001faf f i AccessBridgeMessageQueue.obj
 0001:00000faf       ??_Ebad_alloc@std@@UAEPAXI@Z 10001faf f i AccessBridgeMessageQueue.obj
 0001:00000fd9       ?add@AccessBridgeMessageQueue@@QAE?AW4QueueReturns@@PAVAccessBridgeQueueElement@@@Z 10001fd9 f   AccessBridgeMessageQueue.obj
 0001:00001075       ?getEventsWaiting@AccessBridgeMessageQueue@@QAEHXZ 10002075 f   AccessBridgeMessageQueue.obj
 0001:00001079       ?getRemoveLockSetting@AccessBridgeMessageQueue@@QAEHXZ 10002079 f   AccessBridgeMessageQueue.obj
 0001:0000107d       ?remove@AccessBridgeMessageQueue@@QAE?AW4QueueReturns@@PAPAVAccessBridgeQueueElement@@@Z 1000207d f   AccessBridgeMessageQueue.obj
 0001:00001118       ?setRemoveLock@AccessBridgeMessageQueue@@QAE?AW4QueueReturns@@H@Z 10002118 f   AccessBridgeMessageQueue.obj
 0001:0000112e       ?what@exception@std@@UBEPBDXZ 1000212e f i AccessBridgeMessageQueue.obj
 0001:0000113c       ?initBroadcastMessageIDs@@YAHXZ 1000213c f   AccessBridgeMessages.obj
 0001:0000116e       _Windows_run               1000216e f   AccessBridgeWindowsEntryPoints.obj
 0001:0000117d       _activateAccessibleHyperlink 1000217d f   AccessBridgeWindowsEntryPoints.obj
 0001:000011a4       _addAccessibleSelectionFromContext 100021a4 f   AccessBridgeWindowsEntryPoints.obj
 0001:000011c4       _clearAccessibleSelectionFromContext 100021c4 f   AccessBridgeWindowsEntryPoints.obj
 0001:000011e0       _doAccessibleActions       100021e0 f   AccessBridgeWindowsEntryPoints.obj
 0001:00001207       _getAccessibleActions      10002207 f   AccessBridgeWindowsEntryPoints.obj
 0001:0000122a       _getAccessibleChildFromContext 1000222a f   AccessBridgeWindowsEntryPoints.obj
 0001:0000124f       _getAccessibleContextAt    1000224f f   AccessBridgeWindowsEntryPoints.obj
 0001:00001279       _getAccessibleContextFromHWND 10002279 f   AccessBridgeWindowsEntryPoints.obj
 0001:00001298       _getAccessibleContextInfo  10002298 f   AccessBridgeWindowsEntryPoints.obj
 0001:000012bb       _getAccessibleContextWithFocus 100022bb f   AccessBridgeWindowsEntryPoints.obj
 0001:000012da       _getAccessibleHyperlink    100022da f   AccessBridgeWindowsEntryPoints.obj
 0001:00001301       _getAccessibleHyperlinkCount 10002301 f   AccessBridgeWindowsEntryPoints.obj
 0001:00001321       _getAccessibleHypertext    10002321 f   AccessBridgeWindowsEntryPoints.obj
 0001:00001344       _getAccessibleHypertextExt 10002344 f   AccessBridgeWindowsEntryPoints.obj
 0001:0000136b       _getAccessibleHypertextLinkIndex 1000236b f   AccessBridgeWindowsEntryPoints.obj
 0001:0000138f       _getAccessibleIcons        1000238f f   AccessBridgeWindowsEntryPoints.obj
 0001:000013b2       _getAccessibleKeyBindings  100023b2 f   AccessBridgeWindowsEntryPoints.obj
 0001:000013d5       _getAccessibleParentFromContext 100023d5 f   AccessBridgeWindowsEntryPoints.obj
 0001:000013f6       _getAccessibleRelationSet  100023f6 f   AccessBridgeWindowsEntryPoints.obj
 0001:00001419       _getAccessibleSelectionCountFromContext 10002419 f   AccessBridgeWindowsEntryPoints.obj
 0001:00001439       _getAccessibleSelectionFromContext 10002439 f   AccessBridgeWindowsEntryPoints.obj
 0001:0000145e       _getAccessibleTableCellInfo 1000245e f   AccessBridgeWindowsEntryPoints.obj
 0001:00001488       _getAccessibleTableColumn  10002488 f   AccessBridgeWindowsEntryPoints.obj
 0001:000014ac       _getAccessibleTableColumnDescription 100024ac f   AccessBridgeWindowsEntryPoints.obj
 0001:000014d1       _getAccessibleTableColumnHeader 100024d1 f   AccessBridgeWindowsEntryPoints.obj
 0001:000014f4       _getAccessibleTableColumnSelectionCount 100024f4 f   AccessBridgeWindowsEntryPoints.obj
 0001:00001514       _getAccessibleTableColumnSelections 10002514 f   AccessBridgeWindowsEntryPoints.obj
 0001:0000153b       _getAccessibleTableIndex   1000253b f   AccessBridgeWindowsEntryPoints.obj
 0001:00001563       _getAccessibleTableInfo    10002563 f   AccessBridgeWindowsEntryPoints.obj
 0001:00001586       _getAccessibleTableRow     10002586 f   AccessBridgeWindowsEntryPoints.obj
 0001:000015aa       _getAccessibleTableRowDescription 100025aa f   AccessBridgeWindowsEntryPoints.obj
 0001:000015cf       _getAccessibleTableRowHeader 100025cf f   AccessBridgeWindowsEntryPoints.obj
 0001:000015f2       _getAccessibleTableRowSelectionCount 100025f2 f   AccessBridgeWindowsEntryPoints.obj
 0001:00001612       _getAccessibleTableRowSelections 10002612 f   AccessBridgeWindowsEntryPoints.obj
 0001:00001639       _getAccessibleTextAttributes 10002639 f   AccessBridgeWindowsEntryPoints.obj
 0001:00001660       _getAccessibleTextInfo     10002660 f   AccessBridgeWindowsEntryPoints.obj
 0001:0000168a       _getAccessibleTextItems    1000268a f   AccessBridgeWindowsEntryPoints.obj
 0001:000016b1       _getAccessibleTextLineBounds 100026b1 f   AccessBridgeWindowsEntryPoints.obj
 0001:000016db       _getAccessibleTextRange    100026db f   AccessBridgeWindowsEntryPoints.obj
 0001:00001708       _getAccessibleTextRect     10002708 f   AccessBridgeWindowsEntryPoints.obj
 0001:0000172f       _getAccessibleTextSelectionInfo 1000272f f   AccessBridgeWindowsEntryPoints.obj
 0001:00001752       _getActiveDescendent       10002752 f   AccessBridgeWindowsEntryPoints.obj
 0001:00001773       _getCaretLocation          10002773 f   AccessBridgeWindowsEntryPoints.obj
 0001:0000179a       _getCurrentAccessibleValueFromContext 1000279a f   AccessBridgeWindowsEntryPoints.obj
 0001:000017c1       _getEventsWaiting          100027c1 f   AccessBridgeWindowsEntryPoints.obj
 0001:000017d2       _getHWNDFromAccessibleContext 100027d2 f   AccessBridgeWindowsEntryPoints.obj
 0001:000017f1       _getMaximumAccessibleValueFromContext 100027f1 f   AccessBridgeWindowsEntryPoints.obj
 0001:00001818       _getMinimumAccessibleValueFromContext 10002818 f   AccessBridgeWindowsEntryPoints.obj
 0001:0000183f       _getObjectDepth            1000283f f   AccessBridgeWindowsEntryPoints.obj
 0001:0000185f       _getParentWithRole         1000285f f   AccessBridgeWindowsEntryPoints.obj
 0001:00001884       _getParentWithRoleElseRoot 10002884 f   AccessBridgeWindowsEntryPoints.obj
 0001:000018a9       _getTextAttributesInRange  100028a9 f   AccessBridgeWindowsEntryPoints.obj
 0001:000018d6       _getTopLevelHWND           100028d6 f   AccessBridgeWindowsEntryPoints.obj
 0001:0000190e       _getTopLevelObject         1000290e f   AccessBridgeWindowsEntryPoints.obj
 0001:0000192f       _getVersionInfo            1000292f f   AccessBridgeWindowsEntryPoints.obj
 0001:00001947       _getVirtualAccessibleName  10002947 f   AccessBridgeWindowsEntryPoints.obj
 0001:0000196e       _getVisibleChildren        1000296e f   AccessBridgeWindowsEntryPoints.obj
 0001:00001995       _getVisibleChildrenCount   10002995 f   AccessBridgeWindowsEntryPoints.obj
 0001:000019b4       _isAccessibleChildSelectedFromContext 100029b4 f   AccessBridgeWindowsEntryPoints.obj
 0001:000019d7       _isAccessibleTableColumnSelected 100029d7 f   AccessBridgeWindowsEntryPoints.obj
 0001:000019fa       _isAccessibleTableRowSelected 100029fa f   AccessBridgeWindowsEntryPoints.obj
 0001:00001a1d       _isJavaWindow              10002a1d f   AccessBridgeWindowsEntryPoints.obj
 0001:00001a34       _isSameObject              10002a34 f   AccessBridgeWindowsEntryPoints.obj
 0001:00001a74       _releaseJavaObject         10002a74 f   AccessBridgeWindowsEntryPoints.obj
 0001:00001a90       _removeAccessibleSelectionFromContext 10002a90 f   AccessBridgeWindowsEntryPoints.obj
 0001:00001ab0       _requestFocus              10002ab0 f   AccessBridgeWindowsEntryPoints.obj
 0001:00001acf       _selectAllAccessibleSelectionFromContext 10002acf f   AccessBridgeWindowsEntryPoints.obj
 0001:00001aeb       _selectTextRange           10002aeb f   AccessBridgeWindowsEntryPoints.obj
 0001:00001b12       _setCaretPosition          10002b12 f   AccessBridgeWindowsEntryPoints.obj
 0001:00001b35       _setCaretUpdateFP          10002b35 f   AccessBridgeWindowsEntryPoints.obj
 0001:00001b49       _setFocusGainedFP          10002b49 f   AccessBridgeWindowsEntryPoints.obj
 0001:00001b5d       _setFocusLostFP            10002b5d f   AccessBridgeWindowsEntryPoints.obj
 0001:00001b71       _setJavaShutdownFP         10002b71 f   AccessBridgeWindowsEntryPoints.obj
 0001:00001b85       _setMenuCanceledFP         10002b85 f   AccessBridgeWindowsEntryPoints.obj
 0001:00001b99       _setMenuDeselectedFP       10002b99 f   AccessBridgeWindowsEntryPoints.obj
 0001:00001bad       _setMenuSelectedFP         10002bad f   AccessBridgeWindowsEntryPoints.obj
 0001:00001bc1       _setMouseClickedFP         10002bc1 f   AccessBridgeWindowsEntryPoints.obj
 0001:00001bd5       _setMouseEnteredFP         10002bd5 f   AccessBridgeWindowsEntryPoints.obj
 0001:00001be9       _setMouseExitedFP          10002be9 f   AccessBridgeWindowsEntryPoints.obj
 0001:00001bfd       _setMousePressedFP         10002bfd f   AccessBridgeWindowsEntryPoints.obj
 0001:00001c11       _setMouseReleasedFP        10002c11 f   AccessBridgeWindowsEntryPoints.obj
 0001:00001c25       _setPopupMenuCanceledFP    10002c25 f   AccessBridgeWindowsEntryPoints.obj
 0001:00001c39       _setPopupMenuWillBecomeInvisibleFP 10002c39 f   AccessBridgeWindowsEntryPoints.obj
 0001:00001c4d       _setPopupMenuWillBecomeVisibleFP 10002c4d f   AccessBridgeWindowsEntryPoints.obj
 0001:00001c61       _setPropertyActiveDescendentChangeFP 10002c61 f   AccessBridgeWindowsEntryPoints.obj
 0001:00001c75       _setPropertyCaretChangeFP  10002c75 f   AccessBridgeWindowsEntryPoints.obj
 0001:00001c89       _setPropertyChangeFP       10002c89 f   AccessBridgeWindowsEntryPoints.obj
 0001:00001c9d       _setPropertyChildChangeFP  10002c9d f   AccessBridgeWindowsEntryPoints.obj
 0001:00001cb1       _setPropertyDescriptionChangeFP 10002cb1 f   AccessBridgeWindowsEntryPoints.obj
 0001:00001cc5       _setPropertyNameChangeFP   10002cc5 f   AccessBridgeWindowsEntryPoints.obj
 0001:00001cd9       _setPropertySelectionChangeFP 10002cd9 f   AccessBridgeWindowsEntryPoints.obj
 0001:00001ced       _setPropertyStateChangeFP  10002ced f   AccessBridgeWindowsEntryPoints.obj
 0001:00001d01       _setPropertyTableModelChangeFP 10002d01 f   AccessBridgeWindowsEntryPoints.obj
 0001:00001d15       _setPropertyTextChangeFP   10002d15 f   AccessBridgeWindowsEntryPoints.obj
 0001:00001d29       _setPropertyValueChangeFP  10002d29 f   AccessBridgeWindowsEntryPoints.obj
 0001:00001d3d       _setPropertyVisibleDataChangeFP 10002d3d f   AccessBridgeWindowsEntryPoints.obj
 0001:00001d51       _setTextContents           10002d51 f   AccessBridgeWindowsEntryPoints.obj
 0001:00001d74       ??0WinAccessBridge@@QAE@PAUHINSTANCE__@@@Z 10002d74 f   WinAccessBridge.obj
 0001:00001df2       ??1WinAccessBridge@@QAE@XZ 10002df2 f   WinAccessBridge.obj
 0001:00001eaf       ?JavaVMDestroyed@WinAccessBridge@@QAEXPAUHWND__@@@Z 10002eaf f   WinAccessBridge.obj
 0001:00001f49       ?activateAccessibleHyperlink@WinAccessBridge@@QAEHJ_J0@Z 10002f49 f   WinAccessBridge.obj
 0001:00001fec       ?addAccessibilityEventNotification@WinAccessBridge@@QAEX_J@Z 10002fec f   WinAccessBridge.obj
 0001:00002078       ?addAccessibleSelectionFromContext@WinAccessBridge@@QAEXJ_JH@Z 10003078 f   WinAccessBridge.obj
 0001:000020d8       ?addJavaEventNotification@WinAccessBridge@@QAEX_J@Z 100030d8 f   WinAccessBridge.obj
 0001:00002164       ?clearAccessibleSelectionFromContext@WinAccessBridge@@QAEXJ_J@Z 10003164 f   WinAccessBridge.obj
 0001:000021be       ?doAccessibleActions@WinAccessBridge@@QAEHJ_JPAUAccessibleActionsToDoTag@@PAJ@Z 100031be f   WinAccessBridge.obj
 0001:000022ac       ?getAccessibleActions@WinAccessBridge@@QAEHJ_JPAUAccessibleActionsTag@@@Z 100032ac f   WinAccessBridge.obj
 0001:0000238f       ?getAccessibleChildFromContext@WinAccessBridge@@QAE_JJ_JJ@Z 1000338f f   WinAccessBridge.obj
 0001:00002415       ?getAccessibleContextAt@WinAccessBridge@@QAEHJ_JJJPA_J@Z 10003415 f   WinAccessBridge.obj
 0001:000024bb       ?getAccessibleContextFromHWND@WinAccessBridge@@QAEHPAUHWND__@@PAJPA_J@Z 100034bb f   WinAccessBridge.obj
 0001:000025b6       ?getAccessibleContextInfo@WinAccessBridge@@QAEHJ_JPAUAccessibleContextInfoTag@@@Z 100035b6 f   WinAccessBridge.obj
 0001:00002695       ?getAccessibleContextWithFocus@WinAccessBridge@@QAEHPAUHWND__@@PAJPA_J@Z 10003695 f   WinAccessBridge.obj
 0001:00002735       ?getAccessibleHyperlink@WinAccessBridge@@QAEHJ_JJPAUAccessibleHyperlinkInfoTag@@@Z 10003735 f   WinAccessBridge.obj
 0001:00002813       ?getAccessibleHyperlinkCount@WinAccessBridge@@QAEJJ_J@Z 10003813 f   WinAccessBridge.obj
 0001:000028c4       ?getAccessibleHypertext@WinAccessBridge@@QAEHJ_JPAUAccessibleHypertextInfoTag@@@Z 100038c4 f   WinAccessBridge.obj
 0001:000029a7       ?getAccessibleHypertextExt@WinAccessBridge@@QAEHJ_JJPAUAccessibleHypertextInfoTag@@@Z 100039a7 f   WinAccessBridge.obj
 0001:00002abc       ?getAccessibleHypertextLinkIndex@WinAccessBridge@@QAEJJ_JJ@Z 10003abc f   WinAccessBridge.obj
 0001:00002b75       ?getAccessibleIcons@WinAccessBridge@@QAEHJ_JPAUAccessibleIconsTag@@@Z 10003b75 f   WinAccessBridge.obj
 0001:00002c58       ?getAccessibleKeyBindings@WinAccessBridge@@QAEHJ_JPAUAccessibleKeyBindingsTag@@@Z 10003c58 f   WinAccessBridge.obj
 0001:00002d51       ?getAccessibleParentFromContext@WinAccessBridge@@QAE_JJ_J@Z 10003d51 f   WinAccessBridge.obj
 0001:00002dd0       ?getAccessibleRelationSet@WinAccessBridge@@QAEHJ_JPAUAccessibleRelationSetInfoTag@@@Z 10003dd0 f   WinAccessBridge.obj
 0001:00002eb1       ?getAccessibleSelectionCountFromContext@WinAccessBridge@@QAEHJ_J@Z 10003eb1 f   WinAccessBridge.obj
 0001:00002f18       ?getAccessibleSelectionFromContext@WinAccessBridge@@QAE_JJ_JH@Z 10003f18 f   WinAccessBridge.obj
 0001:00002f89       ?getAccessibleTableCellInfo@WinAccessBridge@@QAEHJ_JJJPAUAccessibleTableCellInfoTag@@@Z 10003f89 f   WinAccessBridge.obj
 0001:00003069       ?getAccessibleTableColumn@WinAccessBridge@@QAEJJ_JJ@Z 10004069 f   WinAccessBridge.obj
 0001:00003111       ?getAccessibleTableColumnDescription@WinAccessBridge@@QAE_JJ_JJ@Z 10004111 f   WinAccessBridge.obj
 0001:000031bf       ?getAccessibleTableColumnHeader@WinAccessBridge@@QAEHJ_JPAUAccessibleTableInfoTag@@@Z 100041bf f   WinAccessBridge.obj
 0001:00003274       ?getAccessibleTableColumnSelectionCount@WinAccessBridge@@QAEJJ_J@Z 10004274 f   WinAccessBridge.obj
 0001:00003310       ?getAccessibleTableColumnSelections@WinAccessBridge@@QAEHJ_JJPAJ@Z 10004310 f   WinAccessBridge.obj
 0001:000033f4       ?getAccessibleTableIndex@WinAccessBridge@@QAEJJ_JJJ@Z 100043f4 f   WinAccessBridge.obj
 0001:000034a8       ?getAccessibleTableInfo@WinAccessBridge@@QAEHJ_JPAUAccessibleTableInfoTag@@@Z 100044a8 f   WinAccessBridge.obj
 0001:00003562       ?getAccessibleTableRow@WinAccessBridge@@QAEJJ_JJ@Z 10004562 f   WinAccessBridge.obj
 0001:0000360a       ?getAccessibleTableRowDescription@WinAccessBridge@@QAE_JJ_JJ@Z 1000460a f   WinAccessBridge.obj
 0001:000036b8       ?getAccessibleTableRowHeader@WinAccessBridge@@QAEHJ_JPAUAccessibleTableInfoTag@@@Z 100046b8 f   WinAccessBridge.obj
 0001:0000376d       ?getAccessibleTableRowSelectionCount@WinAccessBridge@@QAEJJ_J@Z 1000476d f   WinAccessBridge.obj
 0001:00003809       ?getAccessibleTableRowSelections@WinAccessBridge@@QAEHJ_JJPAJ@Z 10004809 f   WinAccessBridge.obj
 0001:000038e8       ?getAccessibleTextAttributes@WinAccessBridge@@QAEHJ_JJPAUAccessibleTextAttributesInfoTag@@@Z 100048e8 f   WinAccessBridge.obj
 0001:0000399c       ?getAccessibleTextInfo@WinAccessBridge@@QAEHJ_JPAUAccessibleTextInfoTag@@JJ@Z 1000499c f   WinAccessBridge.obj
 0001:00003a6a       ?getAccessibleTextItems@WinAccessBridge@@QAEHJ_JPAUAccessibleTextItemsInfoTag@@J@Z 10004a6a f   WinAccessBridge.obj
 0001:00003b4e       ?getAccessibleTextLineBounds@WinAccessBridge@@QAEHJ_JJPAJ1@Z 10004b4e f   WinAccessBridge.obj
 0001:00003bf0       ?getAccessibleTextRange@WinAccessBridge@@QAEHJ_JJJPAGF@Z 10004bf0 f   WinAccessBridge.obj
 0001:00003cce       ?getAccessibleTextRect@WinAccessBridge@@QAEHJ_JPAUAccessibleTextRectInfoTag@@J@Z 10004cce f   WinAccessBridge.obj
 0001:00003d64       ?getAccessibleTextSelectionInfo@WinAccessBridge@@QAEHJ_JPAUAccessibleTextSelectionInfoTag@@@Z 10004d64 f   WinAccessBridge.obj
 0001:00003e0e       ?getActiveDescendent@WinAccessBridge@@QAE_JJ_J@Z 10004e0e f   WinAccessBridge.obj
 0001:00003e8d       ?getCaretLocation@WinAccessBridge@@QAEHJ_JPAUAccessibleTextRectInfoTag@@J@Z 10004e8d f   WinAccessBridge.obj
 0001:00003f23       ?getCurrentAccessibleValueFromContext@WinAccessBridge@@QAEHJ_JPAGF@Z 10004f23 f   WinAccessBridge.obj
 0001:00003fb9       ?getEventsWaiting@WinAccessBridge@@QAEHXZ 10004fb9 f   WinAccessBridge.obj
 0001:00003fc7       ?getHWNDFromAccessibleContext@WinAccessBridge@@QAEPAUHWND__@@J_J@Z 10004fc7 f   WinAccessBridge.obj
 0001:00004048       ?getMaximumAccessibleValueFromContext@WinAccessBridge@@QAEHJ_JPAGF@Z 10005048 f   WinAccessBridge.obj
 0001:000040de       ?getMinimumAccessibleValueFromContext@WinAccessBridge@@QAEHJ_JPAGF@Z 100050de f   WinAccessBridge.obj
 0001:00004174       ?getObjectDepth@WinAccessBridge@@QAEHJ_J@Z 10005174 f   WinAccessBridge.obj
 0001:000041ef       ?getParentWithRole@WinAccessBridge@@QAE_JJ_JPBG@Z 100051ef f   WinAccessBridge.obj
 0001:000042ec       ?getParentWithRoleElseRoot@WinAccessBridge@@QAE_JJ_JPBG@Z 100052ec f   WinAccessBridge.obj
 0001:000043af       ?getTextAttributesInRange@WinAccessBridge@@QAEHJ_JHHPAUAccessibleTextAttributesInfoTag@@PAF@Z 100053af f   WinAccessBridge.obj
 0001:000044bb       ?getTopLevelObject@WinAccessBridge@@QAE_JJ_J@Z 100054bb f   WinAccessBridge.obj
 0001:0000453a       ?getVersionInfo@WinAccessBridge@@QAEHJPAUAccessBridgeVersionInfoTag@@@Z 1000553a f   WinAccessBridge.obj
 0001:000045ee       ?getVirtualAccessibleName@WinAccessBridge@@QAEHJ_JPAGH@Z 100055ee f   WinAccessBridge.obj
 0001:000046cb       ?getVisibleChildren@WinAccessBridge@@QAEHJ_JHPAUVisibleChildenInfoTag@@@Z 100056cb f   WinAccessBridge.obj
 0001:0000477d       ?getVisibleChildrenCount@WinAccessBridge@@QAEHJ_J@Z 1000577d f   WinAccessBridge.obj
 0001:000047f8       ?initWindow@WinAccessBridge@@QAEHXZ 100057f8 f   WinAccessBridge.obj
 0001:00004838       ?isAccessibleChildSelectedFromContext@WinAccessBridge@@QAEHJ_JH@Z 10005838 f   WinAccessBridge.obj
 0001:000048a5       ?isAccessibleTableColumnSelected@WinAccessBridge@@QAEHJ_JJ@Z 100058a5 f   WinAccessBridge.obj
 0001:0000494a       ?isAccessibleTableRowSelected@WinAccessBridge@@QAEHJ_JJ@Z 1000594a f   WinAccessBridge.obj
 0001:000049ef       ?isJavaWindow@WinAccessBridge@@QAEHPAUHWND__@@@Z 100059ef f   WinAccessBridge.obj
 0001:00004a88       ?isSameObject@WinAccessBridge@@QAEHJ_J0@Z 10005a88 f   WinAccessBridge.obj
 0001:00004b43       ?preProcessPackage@WinAccessBridge@@QAEXPADJ@Z 10005b43 f   WinAccessBridge.obj
 0001:00004bd1       ?processPackage@WinAccessBridge@@QAEXPADJ@Z 10005bd1 f   WinAccessBridge.obj
 0001:00005359       ?queuePackage@WinAccessBridge@@QAEHPADJ@Z 10006359 f   WinAccessBridge.obj
 0001:000053b1       ?receiveAQueuedPackage@WinAccessBridge@@QAEHXZ 100063b1 f   WinAccessBridge.obj
 0001:000054a7       ?releaseJavaObject@WinAccessBridge@@QAEXJ_J@Z 100064a7 f   WinAccessBridge.obj
 0001:00005520       ?removeAccessibilityEventNotification@WinAccessBridge@@QAEX_J@Z 10006520 f   WinAccessBridge.obj
 0001:000055ac       ?removeAccessibleSelectionFromContext@WinAccessBridge@@QAEXJ_JH@Z 100065ac f   WinAccessBridge.obj
 0001:0000560c       ?removeJavaEventNotification@WinAccessBridge@@QAEX_J@Z 1000660c f   WinAccessBridge.obj
 0001:00005698       ?rendezvousWithNewJavaDLL@WinAccessBridge@@QAEJPAUHWND__@@J@Z 10006698 f   WinAccessBridge.obj
 0001:00005758       ?requestFocus@WinAccessBridge@@QAEHJ_J@Z 10006758 f   WinAccessBridge.obj
 0001:000057cd       ?selectAllAccessibleSelectionFromContext@WinAccessBridge@@QAEXJ_J@Z 100067cd f   WinAccessBridge.obj
 0001:00005827       ?selectTextRange@WinAccessBridge@@QAEHJ_JHH@Z 10006827 f   WinAccessBridge.obj
 0001:000058ac       ?sendMemoryPackage@WinAccessBridge@@QAEHPADJPAUHWND__@@@Z 100068ac f   WinAccessBridge.obj
 0001:000058fa       ?sendPackage@WinAccessBridge@@QAEXPADJPAUHWND__@@@Z 100068fa f   WinAccessBridge.obj
 0001:00005926       ?setCaretPosition@WinAccessBridge@@QAEHJ_JH@Z 10006926 f   WinAccessBridge.obj
 0001:000059a1       ?setCaretUpdateFP@WinAccessBridge@@QAEXP6AXJ_J0@Z@Z 100069a1 f   WinAccessBridge.obj
 0001:000059b1       ?setFocusGainedFP@WinAccessBridge@@QAEXP6AXJ_J0@Z@Z 100069b1 f   WinAccessBridge.obj
 0001:000059c1       ?setFocusLostFP@WinAccessBridge@@QAEXP6AXJ_J0@Z@Z 100069c1 f   WinAccessBridge.obj
 0001:000059d1       ?setJavaShutdownFP@WinAccessBridge@@QAEXP6AXJ@Z@Z 100069d1 f   WinAccessBridge.obj
 0001:000059e1       ?setMenuCanceledFP@WinAccessBridge@@QAEXP6AXJ_J0@Z@Z 100069e1 f   WinAccessBridge.obj
 0001:000059f1       ?setMenuDeselectedFP@WinAccessBridge@@QAEXP6AXJ_J0@Z@Z 100069f1 f   WinAccessBridge.obj
 0001:00005a01       ?setMenuSelectedFP@WinAccessBridge@@QAEXP6AXJ_J0@Z@Z 10006a01 f   WinAccessBridge.obj
 0001:00005a11       ?setMouseClickedFP@WinAccessBridge@@QAEXP6AXJ_J0@Z@Z 10006a11 f   WinAccessBridge.obj
 0001:00005a21       ?setMouseEnteredFP@WinAccessBridge@@QAEXP6AXJ_J0@Z@Z 10006a21 f   WinAccessBridge.obj
 0001:00005a31       ?setMouseExitedFP@WinAccessBridge@@QAEXP6AXJ_J0@Z@Z 10006a31 f   WinAccessBridge.obj
 0001:00005a41       ?setMousePressedFP@WinAccessBridge@@QAEXP6AXJ_J0@Z@Z 10006a41 f   WinAccessBridge.obj
 0001:00005a51       ?setMouseReleasedFP@WinAccessBridge@@QAEXP6AXJ_J0@Z@Z 10006a51 f   WinAccessBridge.obj
 0001:00005a61       ?setPopupMenuCanceledFP@WinAccessBridge@@QAEXP6AXJ_J0@Z@Z 10006a61 f   WinAccessBridge.obj
 0001:00005a71       ?setPopupMenuWillBecomeInvisibleFP@WinAccessBridge@@QAEXP6AXJ_J0@Z@Z 10006a71 f   WinAccessBridge.obj
 0001:00005a81       ?setPopupMenuWillBecomeVisibleFP@WinAccessBridge@@QAEXP6AXJ_J0@Z@Z 10006a81 f   WinAccessBridge.obj
 0001:00005a91       ?setPropertyActiveDescendentChangeFP@WinAccessBridge@@QAEXP6AXJ_J000@Z@Z 10006a91 f   WinAccessBridge.obj
 0001:00005aa1       ?setPropertyCaretChangeFP@WinAccessBridge@@QAEXP6AXJ_J0HH@Z@Z 10006aa1 f   WinAccessBridge.obj
 0001:00005ab1       ?setPropertyChangeFP@WinAccessBridge@@QAEXP6AXJ_J0PAG11@Z@Z 10006ab1 f   WinAccessBridge.obj
 0001:00005ac1       ?setPropertyChildChangeFP@WinAccessBridge@@QAEXP6AXJ_J000@Z@Z 10006ac1 f   WinAccessBridge.obj
 0001:00005ad1       ?setPropertyDescriptionChangeFP@WinAccessBridge@@QAEXP6AXJ_J0PAG1@Z@Z 10006ad1 f   WinAccessBridge.obj
 0001:00005ae1       ?setPropertyNameChangeFP@WinAccessBridge@@QAEXP6AXJ_J0PAG1@Z@Z 10006ae1 f   WinAccessBridge.obj
 0001:00005af1       ?setPropertySelectionChangeFP@WinAccessBridge@@QAEXP6AXJ_J0@Z@Z 10006af1 f   WinAccessBridge.obj
 0001:00005b01       ?setPropertyStateChangeFP@WinAccessBridge@@QAEXP6AXJ_J0PAG1@Z@Z 10006b01 f   WinAccessBridge.obj
 0001:00005b11       ?setPropertyTableModelChangeFP@WinAccessBridge@@QAEXP6AXJ_J0PAG1@Z@Z 10006b11 f   WinAccessBridge.obj
 0001:00005b21       ?setPropertyTextChangeFP@WinAccessBridge@@QAEXP6AXJ_J0@Z@Z 10006b21 f   WinAccessBridge.obj
 0001:00005b31       ?setPropertyValueChangeFP@WinAccessBridge@@QAEXP6AXJ_J0PAG1@Z@Z 10006b31 f   WinAccessBridge.obj
 0001:00005b41       ?setPropertyVisibleDataChangeFP@WinAccessBridge@@QAEXP6AXJ_J0@Z@Z 10006b41 f   WinAccessBridge.obj
 0001:00005b51       ?setTextContents@WinAccessBridge@@QAEHJ_JPBG@Z 10006b51 f   WinAccessBridge.obj
 0001:00005c14       _AccessBridgeDialogProc@16 10006c14 f   WinAccessBridge.obj
 0001:00005d22       _DllMain@12                10006d22 f   WinAccessBridge.obj
 0001:00005d9f       ??_U@YAPAXI@Z              10006d9f f   MSVCRT:new_array.obj
 0001:00005da8       ??_V@YAXPAX@Z              10006da8 f   MSVCRT:delete_array.obj
 0001:00005db0       __aulldiv                  10006db0 f   MSVCRT:ulldiv.obj
 0001:00005e18       @__security_check_cookie@4 10006e18 f   MSVCRT:secchk.obj
 0001:00005e29       ??3@YAXPAXI@Z              10006e29 f   MSVCRT:delete_scalar_size.obj
 0001:00005e37       ??_Gtype_info@@UAEPAXI@Z   10006e37 f i MSVCRT:std_type_info_static.obj
 0001:00005e37       ??_Etype_info@@UAEPAXI@Z   10006e37 f i MSVCRT:std_type_info_static.obj
 0001:00005e5a       ??2@YAPAXI@Z               10006e5a f   MSVCRT:new_scalar.obj
 0001:00005e90       __alloca_probe             10006e90 f   MSVCRT:chkstk.obj
 0001:00005e90       __chkstk                   10006e90 f   MSVCRT:chkstk.obj
 0001:000061fd       __DllMainCRTStartup@12     100071fd f   MSVCRT:dll_dllmain.obj
 0001:00006220       ??3@YAXPAX@Z               10007220 f   MSVCRT:delete_scalar.obj
 0001:00006225       ___raise_securityfailure   10007225 f   MSVCRT:gs_report.obj
 0001:0000624d       ___report_gsfailure        1000724d f   MSVCRT:gs_report.obj
 0001:00006346       ??0bad_array_new_length@std@@QAE@ABV01@@Z 10007346 f i MSVCRT:throw_bad_alloc.obj
 0001:00006361       ??0bad_array_new_length@std@@QAE@XZ 10007361 f i MSVCRT:throw_bad_alloc.obj
 0001:00006379       ??_Gbad_array_new_length@std@@UAEPAXI@Z 10007379 f i MSVCRT:throw_bad_alloc.obj
 0001:00006379       ??_Ebad_array_new_length@std@@UAEPAXI@Z 10007379 f i MSVCRT:throw_bad_alloc.obj
 0001:000063a6       ?__scrt_throw_std_bad_alloc@@YAXXZ 100073a6 f   MSVCRT:throw_bad_alloc.obj
 0001:000063c3       ?__scrt_throw_std_bad_array_new_length@@YAXXZ 100073c3 f   MSVCRT:throw_bad_alloc.obj
 0001:0000642d       ___security_init_cookie    1000742d f   MSVCRT:gs_support.obj
 0001:00006478       ?__scrt_initialize_type_info@@YAXXZ 10007478 f   MSVCRT:tncleanup.obj
 0001:00006484       ?__scrt_uninitialize_type_info@@YAXXZ 10007484 f   MSVCRT:tncleanup.obj
 0001:00006490       ___local_stdio_scanf_options 10007490 f i MSVCRT:default_local_stdio_options.obj
 0001:00006496       ___scrt_initialize_default_local_stdio_options 10007496 f   MSVCRT:default_local_stdio_options.obj
 0001:000064f7       ___scrt_acquire_startup_lock 100074f7 f   MSVCRT:utility.obj
 0001:00006529       ___scrt_dllmain_after_initialize_c 10007529 f   MSVCRT:utility.obj
 0001:00006554       ___scrt_dllmain_before_initialize_c 10007554 f   MSVCRT:utility.obj
 0001:00006562       ___scrt_dllmain_crt_thread_attach 10007562 f   MSVCRT:utility.obj
 0001:00006581       ___scrt_dllmain_crt_thread_detach 10007581 f   MSVCRT:utility.obj
 0001:0000658e       ___scrt_dllmain_exception_filter 1000758e f   MSVCRT:utility.obj
 0001:000065c2       ___scrt_dllmain_uninitialize_c 100075c2 f   MSVCRT:utility.obj
 0001:000065e5       ___scrt_dllmain_uninitialize_critical 100075e5 f   MSVCRT:utility.obj
 0001:000065f2       ___scrt_initialize_crt     100075f2 f   MSVCRT:utility.obj
 0001:0000662b       ___scrt_initialize_onexit_tables 1000762b f   MSVCRT:utility.obj
 0001:000066b2       ___scrt_is_nonwritable_in_current_image 100076b2 f   MSVCRT:utility.obj
 0001:00006746       ___scrt_release_startup_lock 10007746 f   MSVCRT:utility.obj
 0001:00006763       ___scrt_uninitialize_crt   10007763 f   MSVCRT:utility.obj
 0001:0000678b       ___scrt_get_dyn_tls_init_callback 1000778b f   MSVCRT:dyn_tls_init.obj
 0001:00006791       ___scrt_fastfail           10007791 f   MSVCRT:utility_desktop.obj
 0001:000068ab       __crt_debugger_hook        100078ab f   MSVCRT:utility_desktop.obj
 0001:000068b3       __RTC_Initialize           100078b3 f   MSVCRT:initsect.obj
 0001:000068df       __RTC_Terminate            100078df f   MSVCRT:initsect.obj
 0001:00006910       __SEH_prolog4              10007910 f   MSVCRT:sehprolg4.obj
 0001:00006954       __SEH_epilog4              10007954 f   MSVCRT:sehprolg4.obj
 0001:00006968       __except_handler4          10007968 f   MSVCRT:chandler4gs.obj
 0001:00006997       ___isa_available_init      10007997 f   MSVCRT:cpu_disp.obj
 0001:00006b67       __get_startup_argv_mode    10007b67 f   MSVCRT:argv_mode.obj
 0001:00006b6b       ___scrt_is_ucrt_dll_in_use 10007b6b f   MSVCRT:ucrt_detection.obj
 0001:00006b77       _memcpy                    10007b77 f   vcruntime:VCRUNTIME140.dll
 0001:00006b7d       _memset                    10007b7d f   vcruntime:VCRUNTIME140.dll
 0001:00006b83       ___std_exception_copy      10007b83 f   vcruntime:VCRUNTIME140.dll
 0001:00006b89       ___std_exception_destroy   10007b89 f   vcruntime:VCRUNTIME140.dll
 0001:00006b8f       __CxxThrowException@8      10007b8f f   vcruntime:VCRUNTIME140.dll
 0001:00006b95       ___std_type_info_destroy_list 10007b95 f   vcruntime:VCRUNTIME140.dll
 0001:00006b9b       __except_handler4_common   10007b9b f   vcruntime:VCRUNTIME140.dll
 0001:00006ba1       _strlen                    10007ba1 f   ucrt:api-ms-win-crt-string-l1-1-0.dll
 0001:00006ba7       _strcmp                    10007ba7 f   ucrt:api-ms-win-crt-string-l1-1-0.dll
 0001:00006bad       _strcpy                    10007bad f   ucrt:api-ms-win-crt-string-l1-1-0.dll
 0001:00006bb3       _free                      10007bb3 f   ucrt:api-ms-win-crt-heap-l1-1-0.dll
 0001:00006bb9       _malloc                    10007bb9 f   ucrt:api-ms-win-crt-heap-l1-1-0.dll
 0001:00006bbf       __callnewh                 10007bbf f   ucrt:api-ms-win-crt-heap-l1-1-0.dll
 0001:00006bc5       __initterm                 10007bc5 f   ucrt:api-ms-win-crt-runtime-l1-1-0.dll
 0001:00006bcb       __initterm_e               10007bcb f   ucrt:api-ms-win-crt-runtime-l1-1-0.dll
 0001:00006bd1       __seh_filter_dll           10007bd1 f   ucrt:api-ms-win-crt-runtime-l1-1-0.dll
 0001:00006bd7       __configure_narrow_argv    10007bd7 f   ucrt:api-ms-win-crt-runtime-l1-1-0.dll
 0001:00006bdd       __initialize_narrow_environment 10007bdd f   ucrt:api-ms-win-crt-runtime-l1-1-0.dll
 0001:00006be3       __initialize_onexit_table  10007be3 f   ucrt:api-ms-win-crt-runtime-l1-1-0.dll
 0001:00006be9       __execute_onexit_table     10007be9 f   ucrt:api-ms-win-crt-runtime-l1-1-0.dll
 0001:00006bef       __cexit                    10007bef f   ucrt:api-ms-win-crt-runtime-l1-1-0.dll
 0001:00006bf5       _IsProcessorFeaturePresent@4 10007bf5 f   kernel32:KERNEL32.dll
 0001:00006bfb       ___vcrt_thread_detach      10007bfb f   MSVCRT:ucrt_stubs.obj
 0001:00006bfb       ___acrt_initialize         10007bfb f   MSVCRT:ucrt_stubs.obj
 0001:00006bfb       ___vcrt_initialize         10007bfb f   MSVCRT:ucrt_stubs.obj
 0001:00006bfb       ___scrt_stub_for_acrt_thread_attach 10007bfb f   MSVCRT:ucrt_stubs.obj
 0001:00006bfb       ___vcrt_uninitialize_critical 10007bfb f   MSVCRT:ucrt_stubs.obj
 0001:00006bfb       ___scrt_stub_for_acrt_uninitialize_critical 10007bfb f   MSVCRT:ucrt_stubs.obj
 0001:00006bfb       ___scrt_stub_for_acrt_initialize 10007bfb f   MSVCRT:ucrt_stubs.obj
 0001:00006bfb       ___acrt_uninitialize_critical 10007bfb f   MSVCRT:ucrt_stubs.obj
 0001:00006bfb       ___acrt_uninitialize       10007bfb f   MSVCRT:ucrt_stubs.obj
 0001:00006bfb       ___acrt_thread_detach      10007bfb f   MSVCRT:ucrt_stubs.obj
 0001:00006bfb       ___scrt_stub_for_acrt_thread_detach 10007bfb f   MSVCRT:ucrt_stubs.obj
 0001:00006bfb       ___vcrt_thread_attach      10007bfb f   MSVCRT:ucrt_stubs.obj
 0001:00006bfb       ___scrt_stub_for_acrt_uninitialize 10007bfb f   MSVCRT:ucrt_stubs.obj
 0001:00006bfb       ___acrt_thread_attach      10007bfb f   MSVCRT:ucrt_stubs.obj
 0001:00006bfb       ___vcrt_uninitialize       10007bfb f   MSVCRT:ucrt_stubs.obj
 0001:00006bfe       __is_c_termination_complete 10007bfe f   MSVCRT:ucrt_stubs.obj
 0001:00006bfe       ___scrt_stub_for_is_c_termination_complete 10007bfe f   MSVCRT:ucrt_stubs.obj
 0001:00006c01       __filter_x86_sse2_floating_point_exception 10007c01 f   MSVCRT:x86_exception_filter.obj
 0001:00006c01       __filter_x86_sse2_floating_point_exception_default 10007c01 f   MSVCRT:x86_exception_filter.obj
 0002:00000000       __imp__GetLastError@0      10008000     kernel32:KERNEL32.dll
 0002:00000004       __imp__GetSystemTimeAsFileTime@4 10008004     kernel32:KERNEL32.dll
 0002:00000008       __imp__CloseHandle@4       10008008     kernel32:KERNEL32.dll
 0002:0000000c       __imp__EnterCriticalSection@4 1000800c     kernel32:KERNEL32.dll
 0002:00000010       __imp__LeaveCriticalSection@4 10008010     kernel32:KERNEL32.dll
 0002:00000014       __imp__MapViewOfFile@20    10008014     kernel32:KERNEL32.dll
 0002:00000018       __imp__UnmapViewOfFile@4   10008018     kernel32:KERNEL32.dll
 0002:0000001c       __imp__CreateFileMappingA@24 1000801c     kernel32:KERNEL32.dll
 0002:00000020       __imp__InitializeCriticalSection@4 10008020     kernel32:KERNEL32.dll
 0002:00000024       __imp__IsDebuggerPresent@0 10008024     kernel32:KERNEL32.dll
 0002:00000028       __imp__InitializeSListHead@4 10008028     kernel32:KERNEL32.dll
 0002:0000002c       __imp__GetCurrentThreadId@0 1000802c     kernel32:KERNEL32.dll
 0002:00000030       __imp__GetCurrentProcessId@0 10008030     kernel32:KERNEL32.dll
 0002:00000034       __imp__QueryPerformanceCounter@4 10008034     kernel32:KERNEL32.dll
 0002:00000038       __imp__IsProcessorFeaturePresent@4 10008038     kernel32:KERNEL32.dll
 0002:0000003c       __imp__TerminateProcess@8  1000803c     kernel32:KERNEL32.dll
 0002:00000040       __imp__GetCurrentProcess@0 10008040     kernel32:KERNEL32.dll
 0002:00000044       __imp__SetUnhandledExceptionFilter@4 10008044     kernel32:KERNEL32.dll
 0002:00000048       __imp__UnhandledExceptionFilter@4 10008048     kernel32:KERNEL32.dll
 0002:0000004c       \177KERNEL32_NULL_THUNK_DATA 1000804c     kernel32:KERNEL32.dll
 0002:00000050       __imp__ShowWindow@8        10008050     user32:USER32.dll
 0002:00000054       __imp__DestroyWindow@4     10008054     user32:USER32.dll
 0002:00000058       __imp__PostMessageA@16     10008058     user32:USER32.dll
 0002:0000005c       __imp__SendMessageA@16     1000805c     user32:USER32.dll
 0002:00000060       __imp__GetParent@4         10008060     user32:USER32.dll
 0002:00000064       __imp__GetWindowLongA@8    10008064     user32:USER32.dll
 0002:00000068       __imp__IsWindow@4          10008068     user32:USER32.dll
 0002:0000006c       __imp__RegisterWindowMessageA@4 1000806c     user32:USER32.dll
 0002:00000070       __imp__SendMessageTimeoutA@28 10008070     user32:USER32.dll
 0002:00000074       __imp__CreateDialogParamA@20 10008074     user32:USER32.dll
 0002:00000078       \177USER32_NULL_THUNK_DATA 10008078     user32:USER32.dll
 0002:0000007c       __imp___except_handler4_common 1000807c     vcruntime:VCRUNTIME140.dll
 0002:00000080       __imp___CxxThrowException@8 10008080     vcruntime:VCRUNTIME140.dll
 0002:00000084       __imp____std_exception_destroy 10008084     vcruntime:VCRUNTIME140.dll
 0002:00000088       __imp____std_exception_copy 10008088     vcruntime:VCRUNTIME140.dll
 0002:0000008c       __imp____std_type_info_destroy_list 1000808c     vcruntime:VCRUNTIME140.dll
 0002:00000090       __imp__memset              10008090     vcruntime:VCRUNTIME140.dll
 0002:00000094       __imp__memcpy              10008094     vcruntime:VCRUNTIME140.dll
 0002:00000098       \177VCRUNTIME140_NULL_THUNK_DATA 10008098     vcruntime:VCRUNTIME140.dll
 0002:0000009c       __imp__getenv              1000809c     ucrt:api-ms-win-crt-environment-l1-1-0.dll
 0002:000000a0       \177api-ms-win-crt-environment-l1-1-0_NULL_THUNK_DATA 100080a0     ucrt:api-ms-win-crt-environment-l1-1-0.dll
 0002:000000a4       __imp__free                100080a4     ucrt:api-ms-win-crt-heap-l1-1-0.dll
 0002:000000a8       __imp___callnewh           100080a8     ucrt:api-ms-win-crt-heap-l1-1-0.dll
 0002:000000ac       __imp__malloc              100080ac     ucrt:api-ms-win-crt-heap-l1-1-0.dll
 0002:000000b0       \177api-ms-win-crt-heap-l1-1-0_NULL_THUNK_DATA 100080b0     ucrt:api-ms-win-crt-heap-l1-1-0.dll
 0002:000000b4       __imp___seh_filter_dll     100080b4     ucrt:api-ms-win-crt-runtime-l1-1-0.dll
 0002:000000b8       __imp___configure_narrow_argv 100080b8     ucrt:api-ms-win-crt-runtime-l1-1-0.dll
 0002:000000bc       __imp___initialize_narrow_environment 100080bc     ucrt:api-ms-win-crt-runtime-l1-1-0.dll
 0002:000000c0       __imp___initterm           100080c0     ucrt:api-ms-win-crt-runtime-l1-1-0.dll
 0002:000000c4       __imp___execute_onexit_table 100080c4     ucrt:api-ms-win-crt-runtime-l1-1-0.dll
 0002:000000c8       __imp___cexit              100080c8     ucrt:api-ms-win-crt-runtime-l1-1-0.dll
 0002:000000cc       __imp___initterm_e         100080cc     ucrt:api-ms-win-crt-runtime-l1-1-0.dll
 0002:000000d0       __imp___initialize_onexit_table 100080d0     ucrt:api-ms-win-crt-runtime-l1-1-0.dll
 0002:000000d4       \177api-ms-win-crt-runtime-l1-1-0_NULL_THUNK_DATA 100080d4     ucrt:api-ms-win-crt-runtime-l1-1-0.dll
 0002:000000d8       __imp____acrt_iob_func     100080d8     ucrt:api-ms-win-crt-stdio-l1-1-0.dll
 0002:000000dc       __imp____stdio_common_vfprintf 100080dc     ucrt:api-ms-win-crt-stdio-l1-1-0.dll
 0002:000000e0       __imp__fclose              100080e0     ucrt:api-ms-win-crt-stdio-l1-1-0.dll
 0002:000000e4       __imp____stdio_common_vsprintf 100080e4     ucrt:api-ms-win-crt-stdio-l1-1-0.dll
 0002:000000e8       __imp__fopen               100080e8     ucrt:api-ms-win-crt-stdio-l1-1-0.dll
 0002:000000ec       \177api-ms-win-crt-stdio-l1-1-0_NULL_THUNK_DATA 100080ec     ucrt:api-ms-win-crt-stdio-l1-1-0.dll
 0002:000000f0       __imp__wcsncpy             100080f0     ucrt:api-ms-win-crt-string-l1-1-0.dll
 0002:000000f4       __imp__strcpy              100080f4     ucrt:api-ms-win-crt-string-l1-1-0.dll
 0002:000000f8       __imp__strncpy             100080f8     ucrt:api-ms-win-crt-string-l1-1-0.dll
 0002:000000fc       __imp__strlen              100080fc     ucrt:api-ms-win-crt-string-l1-1-0.dll
 0002:00000100       __imp__strcmp              10008100     ucrt:api-ms-win-crt-string-l1-1-0.dll
 0002:00000104       \177api-ms-win-crt-string-l1-1-0_NULL_THUNK_DATA 10008104     ucrt:api-ms-win-crt-string-l1-1-0.dll
 0002:00000108       ___guard_check_icall_fptr  10008108     MSVCRT:guard_support.obj
 0002:0000010c       ___xc_a                    1000810c     MSVCRT:initializers.obj
 0002:00000110       ___xc_z                    10008110     MSVCRT:initializers.obj
 0002:00000114       ___xi_a                    10008114     MSVCRT:initializers.obj
 0002:00000118       ___xi_z                    10008118     MSVCRT:initializers.obj
 0002:0000011c       ___xp_a                    1000811c     MSVCRT:initializers.obj
 0002:00000120       ___xp_z                    10008120     MSVCRT:initializers.obj
 0002:00000124       ___xt_a                    10008124     MSVCRT:initializers.obj
 0002:00000128       ___xt_z                    10008128     MSVCRT:initializers.obj
 0002:00000130       ??_C@_0BJ@FKCDJFDK@JAVA_ACCESSBRIDGE_LOGDIR@ 10008130     AccessBridgeDebug.obj
 0002:0000014c       ??_C@_04FPOLKAEB@?4log@    1000814c     AccessBridgeDebug.obj
 0002:00000154       ??_C@_01NOFIACDB@w@        10008154     AccessBridgeDebug.obj
 0002:00000158       ??_C@_04EINJHBMM@?6?$CFs?6@ 10008158     AccessBridgeDebug.obj
 0002:00000160       ??_C@_0BH@PPBGFLKL@Could?5not?5open?5file?5?$CFs@ 10008160     AccessBridgeDebug.obj
 0002:00000178       ??_C@_07IBOBEFLP@?$FL?$CFllu?$FN?5@ 10008178     AccessBridgeDebug.obj
 0002:00000180       ??_C@_02PCIJFNDE@?$AN?6@   10008180     AccessBridgeDebug.obj
 0002:00000184       ??_C@_0BH@BLGOOJIK@AccessBridge?9?$CFp?9?$CFp?4mmf@ 10008184     AccessBridgeJavaVMInstance.obj
 0002:0000019c       ??_C@_03DJNNCAJF@OK?$DP@   1000819c     AccessBridgeJavaVMInstance.obj
 0002:000001a0       ??_C@_03ONJMBPEK@OK?$CB@   100081a0     AccessBridgeJavaVMInstance.obj
 0002:000001a4       ??_C@_0CP@JIGBIHFH@?$FLINFO?$FN?3?5In?5AccessBridgeVMInstan@ 100081a4     AccessBridgeJavaVMInstance.obj
 0002:000001d4       ??_C@_0CH@KAGNBCII@?$FLINFO?$FN?3?5?5?5?5?5javaAccessBridgeWin@ 100081d4     AccessBridgeJavaVMInstance.obj
 0002:000001fc       ??_C@_0CC@NKGMANMJ@?$FLINFO?$FN?3?5In?5findAccessBridgeWind@ 100081fc     AccessBridgeJavaVMInstance.obj
 0002:00000220       ??_C@_0CK@NBPNOPCH@?$FLINFO?$FN?3?5In?5findABJavaInstanceFr@ 10008220     AccessBridgeJavaVMInstance.obj
 0002:00000250       ??_7exception@std@@6B@     10008250     AccessBridgeMessageQueue.obj
 0002:00000258       ??_C@_0BC@EOODALEL@Unknown?5exception@ 10008258     AccessBridgeMessageQueue.obj
 0002:00000270       ??_7bad_alloc@std@@6B@     10008270     AccessBridgeMessageQueue.obj
 0002:00000278       ??_C@_0P@GHFPNOJB@bad?5allocation@ 10008278     AccessBridgeMessageQueue.obj
 0002:00000288       ??_C@_0CN@EPCNBBKD@?$FLINFO?$FN?3?5?5?5in?5AccessBridgeMessag@ 10008288     AccessBridgeMessageQueue.obj
 0002:000002b8       ??_C@_0BM@FHOEMINC@?$FLINFO?$FN?3?5?5?5?5?5queue?5size?5?$DN?5?$CFd@ 100082b8     AccessBridgeMessageQueue.obj
 0002:000002d4       ??_C@_0DF@PKPPNDEN@?$FLWARN?$FN?3?5?5?5?5?5queue?5was?5locked?$DL?5r@ 100082d4     AccessBridgeMessageQueue.obj
 0002:0000030c       ??_C@_0CF@CAPEOLCL@?$FLINFO?$FN?3?5?5?5?5?5adding?5element?5to?5q@ 1000830c     AccessBridgeMessageQueue.obj
 0002:00000334       ??_C@_0DL@IILCMNMG@?$FLINFO?$FN?3?5?5?5?5?5returning?5from?5Acce@ 10008334     AccessBridgeMessageQueue.obj
 0002:00000370       ??_C@_0DA@NHLJEKKG@?$FLINFO?$FN?3?5?5?5in?5AccessBridgeMessag@ 10008370     AccessBridgeMessageQueue.obj
 0002:000003a0       ??_C@_0CJ@FBOCEMKO@?$FLINFO?$FN?3?5?5?5?5?5removing?5element?5fr@ 100083a0     AccessBridgeMessageQueue.obj
 0002:000003cc       ??_C@_0DO@NEJIEHGM@?$FLINFO?$FN?3?5?5?5?5?5returning?5from?5Acce@ 100083cc     AccessBridgeMessageQueue.obj
 0002:0000040c       ??_C@_0BM@BIAOFPJG@AccessBridge?9FromJava?9Hello@ 1000840c     AccessBridgeMessages.obj
 0002:00000428       ??_C@_0BP@OELHMMDF@AccessBridge?9FromWindows?9Hello@ 10008428     AccessBridgeMessages.obj
 0002:00000448       ??_C@_0EC@DLPGLEGA@?$AN?6AccessBridgeWindowsEntryPoint@ 10008448     AccessBridgeWindowsEntryPoints.obj
 0002:0000048c       ??_C@_0BG@GGFIABLO@windows_access_bridge@ 1000848c     WinAccessBridge.obj
 0002:000004a4       ??_C@_0BL@GLCNGDJJ@?$FLINFO?$FN?3?5DLL_PROCESS_ATTACH@ 100084a4     WinAccessBridge.obj
 0002:000004c0       ??_C@_0EG@HHOMJPNP@?$FLINFO?$FN?3?5?$CK?$CK?$CK?5AccessBridgeDialogP@ 100084c0     WinAccessBridge.obj
 0002:00000508       ??_C@_0CP@LHINEKAP@?$FLINFO?$FN?3?5AccessBridgeDialogProc?5@ 10008508     WinAccessBridge.obj
 0002:00000538       ??_C@_0EH@MDELPMEJ@?$FLINFO?$FN?3?5AccessBridgeDialogProc?5@ 10008538     WinAccessBridge.obj
 0002:00000580       ??_C@_0DP@HBEMDAPF@?$FLINFO?$FN?3?5AccessBridgeDialogProc?5@ 10008580     WinAccessBridge.obj
 0002:000005c0       ??_C@_0EH@MPLEACPJ@?$FLINFO?$FN?3?5AccessBridgeDialogProc?5@ 100085c0     WinAccessBridge.obj
 0002:00000608       ??_C@_0EG@GGGHDKAD@?$FLINFO?$FN?3?5?$CK?$CK?$CK?$CK?$CK?5AccessBridgeDialo@ 10008608     WinAccessBridge.obj
 0002:00000650       ??_C@_0DE@BGNNIIOB@?$FLINFO?$FN?3?5?5?5javaVMs?5chain?5in?5use?0@ 10008650     WinAccessBridge.obj
 0002:00000684       ??_C@_0CC@NEJJLLGC@?$FLINFO?$FN?3?5?5?5calling?5javaVMDestroy@ 10008684     WinAccessBridge.obj
 0002:000006a8       ??_C@_0FG@BHPCMIAO@?$FLINFO?$FN?3?5AccessBridgeDialogProc?5@ 100086a8     WinAccessBridge.obj
 0002:00000700       ??_C@_0BN@FIPGEIKI@?$FLINFO?$FN?3?5WinAccessBridge?5ctor@ 10008700     WinAccessBridge.obj
 0002:00000720       ??_C@_0DE@JFKNENGC@?$FLINFO?$FN?3?5?$CK?$CK?$CK?$CK?$CKin?5WinAccessBridge@ 10008720     WinAccessBridge.obj
 0002:00000754       ??_C@_0CG@EDMKMONP@?$FLINFO?$FN?3?5?5?5telling?5?$CFp?5we?8re?5goin@ 10008754     WinAccessBridge.obj
 0002:0000077c       ??_C@_0DB@CFPLAPDG@?$FLINFO?$FN?3?5?5?5finished?5telling?5JVMs@ 1000877c     WinAccessBridge.obj
 0002:000007b0       ??_C@_0EE@GBJFCFOA@?$FLINFO?$FN?3?5?5?5finished?5deleting?5eve@ 100087b0     WinAccessBridge.obj
 0002:000007f4       ??_C@_0BP@EBFMIPOK@?$FLINFO?$FN?3?5GOODBYE?5CRUEL?5WORLD?4?4?4@ 100087f4     WinAccessBridge.obj
 0002:00000814       ??_C@_0BJ@LMONFDOG@ACCESSBRIDGESTATUSWINDOW@ 10008814     WinAccessBridge.obj
 0002:00000830       ??_C@_0DN@NNELAOKC@?$FLINFO?$FN?3?5in?5WinAccessBridge?3?3ren@ 10008830     WinAccessBridge.obj
 0002:00000870       ??_C@_0CJ@LMLGKPGD@?$FLINFO?$FN?3?5?5?5Setting?5Java?5event?5ma@ 10008870     WinAccessBridge.obj
 0002:0000089c       ??_C@_0DC@IJKHOBEO@?$FLINFO?$FN?3?5?5?5Setting?5Accessibility@ 1000889c     WinAccessBridge.obj
 0002:000008d0       ??_C@_0DN@ECLBFGAO@?$FLERROR?$FN?3?5Failed?5to?5initiate?5IPC@ 100088d0     WinAccessBridge.obj
 0002:00000910       ??_C@_0DG@OEMNKFJP@?$FLINFO?$FN?3?5?5?5Success?$CB?$CB?5?5We?5rendezv@ 10008910     WinAccessBridge.obj
 0002:00000948       ??_C@_0DK@BLMJEFJH@?$FLERROR?$FN?3?5sending?5memory?5package@ 10008948     WinAccessBridge.obj
 0002:00000984       ??_C@_0DC@BABNPCOM@?$FLINFO?$FN?3?5?5in?5WinAccessBridge?3?3qu@ 10008984     WinAccessBridge.obj
 0002:000009b8       ??_C@_0DE@NOAFOCML@?$FLINFO?$FN?3?5in?5WinAccessBridge?3?3rec@ 100089b8     WinAccessBridge.obj
 0002:000009ec       ??_C@_0BM@KNOOFOHJ@?$FLINFO?$FN?3?5?5dequeueing?5message@ 100089ec     WinAccessBridge.obj
 0002:00000a08       ??_C@_0CD@GBHFIMOB@?$FLERROR?$FN?3?5Queue?5seems?5to?5be?5brok@ 10008a08     WinAccessBridge.obj
 0002:00000a2c       ??_C@_0CA@LFELFFDM@?$FLINFO?$FN?3?5?5found?5one?$DL?5sending?5it?$CB@ 10008a2c     WinAccessBridge.obj
 0002:00000a4c       ??_C@_0BP@ENBFDBDP@?$FLWARN?$FN?3?5?5?5ODD?4?4?4?5element?5?$DN?$DN?50?$CB@ 10008a4c     WinAccessBridge.obj
 0002:00000a6c       ??_C@_0CP@OIAJKCPF@?$FLWARN?$FN?3?5?5Queue?5in?5use?0?5will?5try@ 10008a6c     WinAccessBridge.obj
 0002:00000a9c       ??_C@_0DH@KAJCMPPF@?$FLWARN?$FN?3?5?5unable?5to?5dequeue?5mess@ 10008a9c     WinAccessBridge.obj
 0002:00000ad4       ??_C@_0CO@KCIANNAF@?$FLINFO?$FN?3?5PreProcessing?5package?5s@ 10008ad4     WinAccessBridge.obj
 0002:00000b08       ??_C@_0EF@DFMGOCJF@?$FLERROR?$FN?3?5?5?5processing?5FAILED?$CB?$CB?5@ 10008b08     WinAccessBridge.obj
 0002:00000b50       ??_C@_0CL@HBCKEPEE@?$FLINFO?$FN?3?5?5?5?5package?5preprocessin@ 10008b50     WinAccessBridge.obj
 0002:00000b7c       ??_C@_0DM@CCADHAH@?$FLINFO?$FN?3?5WinAccessBridge?3?3Proces@ 10008b7c     WinAccessBridge.obj
 0002:00000bb8       ??_C@_0CI@KAACKIJC@?$FLINFO?$FN?3?5?5?5?5type?5?$DN?$DN?5cJavaShutdow@ 10008bb8     WinAccessBridge.obj
 0002:00000be0       ??_C@_0CE@KGDIDFJM@?$FLINFO?$FN?3?5?5?5?5event?5callback?5compl@ 10008be0     WinAccessBridge.obj
 0002:00000c04       ??_C@_0BI@MGOIGNJM@?$FLINFO?$FN?3?5?5?5?5event?5fired?$CB@ 10008c04     WinAccessBridge.obj
 0002:00000c20       ??_C@_0EC@JELBKKLB@?$FLERROR?$FN?3?5?5?5?5processing?5FAILED?$CB?$CB@ 10008c20     WinAccessBridge.obj
 0002:00000c64       ??_C@_0CM@OIHFPHBP@?$FLINFO?$FN?3?5?5?5?5begin?5callback?5to?5AT@ 10008c64     WinAccessBridge.obj
 0002:00000c90       ??_C@_0EB@PCOLNIOI@?$FLERROR?$FN?3?5?5?5processing?5FAILED?$CB?$CB?5@ 10008c90     WinAccessBridge.obj
 0002:00000cd8       ??_C@_0EG@DADDGPDA@?$FLERROR?$FN?3?5?5?5?5processing?5FAILED?$CB?$CB@ 10008cd8     WinAccessBridge.obj
 0002:00000d20       ??_C@_0CI@PMGDCMNI@?$FLINFO?$FN?3?5?5?5?5package?5processing?5c@ 10008d20     WinAccessBridge.obj
 0002:00000d48       ??_C@_0DD@EDMANGOO@?$FLINFO?$FN?3?5?$CK?$CK?$CK?$CK?$CK?5WinAccessBridge?3?3@ 10008d48     WinAccessBridge.obj
 0002:00000d7c       ??_C@_0CP@IIHJFGGB@?$FLINFO?$FN?3?5?5?5data?5structures?5succe@ 10008d7c     WinAccessBridge.obj
 0002:00000dac       ??_C@_0DB@JABMCGEJ@?$FLERROR?$FN?3?5couldn?8t?5find?5matching@ 10008dac     WinAccessBridge.obj
 0002:00000de0       ??_C@_0DJ@EFGAHBMH@?$FLINFO?$FN?3?5WinAccessBridge?3?3releas@ 10008de0     WinAccessBridge.obj
 0002:00000e1c       ??_C@_0CO@GDCOMIDN@?$FLINFO?$FN?3?5WinAccessBridge?3?3getVer@ 10008e1c     WinAccessBridge.obj
 0002:00000e50       ??_C@_0IH@JNMBAFNI@?$FLINFO?$FN?3?5?5?5VMversion?3?5?$CFls?6?5?5?5?5?5?5@ 10008e50     WinAccessBridge.obj
 0002:00000ed8       ??_C@_0CJ@MFBANPLF@?$FLINFO?$FN?3?5In?5WinAccessBridge?3?3isJ@ 10008ed8     WinAccessBridge.obj
 0002:00000f04       ??_C@_0CK@OIADIKJK@?$FLINFO?$FN?3?5WinAccessBridge?3?3isJava@ 10008f04     WinAccessBridge.obj
 0002:00000f30       ??_C@_0DJ@GDIICFAI@?$FLINFO?$FN?3?5WinAccessBridge?3?3isSame@ 10008f30     WinAccessBridge.obj
 0002:00000f70       ??_C@_0EF@JHJAECO@?$FLINFO?$FN?3?5?5?5WinAccessBridge?3?3isSa@ 10008f70     WinAccessBridge.obj
 0002:00000fb8       ??_C@_0EL@EGCPHNBB@?$FLINFO?$FN?3?5?5?5WinAccessBridge?3?3isSa@ 10008fb8     WinAccessBridge.obj
 0002:00001008       ??_C@_0FE@JNIGOBOL@?$FLERROR?$FN?3?5?5?5WinAccessBridge?3?3isS@ 10009008     WinAccessBridge.obj
 0002:0000105c       ??_C@_0DM@KHCMPGEG@?$FLINFO?$FN?3?5WinAccessBridge?3?3getAcc@ 1000905c     WinAccessBridge.obj
 0002:00001098       ??_C@_0DA@KDJKNLAN@?$FLINFO?$FN?3?5?5?5?5?5current?9?$DOvmID?5?$DN?5?$CFX?0@ 10009098     WinAccessBridge.obj
 0002:000010c8       ??_C@_0CP@IJNFIHAG@?$FLINFO?$FN?3?5?5?5?5?5pkg?9?$DOrAccessibleCon@ 100090c8     WinAccessBridge.obj
 0002:000010f8       ??_C@_0DJ@FFBPMFOM@?$FLERROR?$FN?3?5getAccessibleContextFr@ 100090f8     WinAccessBridge.obj
 0002:00001134       ??_C@_0DO@IIGOCPCC@?$FLERROR?$FN?3?5getAccessibleContextFr@ 10009134     WinAccessBridge.obj
 0002:00001174       ??_C@_0DL@KEEIEGBJ@?$FLINFO?$FN?3?5?5?5in?5WinAccessBridge?3?3g@ 10009174     WinAccessBridge.obj
 0002:000011b0       ??_C@_0EA@HDGDGEMM@?$FLINFO?$FN?3?5WinAccessBridge?3?3getHWN@ 100091b0     WinAccessBridge.obj
 0002:000011f0       ??_C@_0EA@FHJPOEHJ@?$FLINFO?$FN?3?5WinAccessBridge?3?3getAcc@ 100091f0     WinAccessBridge.obj
 0002:00001230       ??_C@_0EB@HKEAOAKG@?$FLINFO?$FN?3?5WinAccessBridge?3?3getAcc@ 10009230     WinAccessBridge.obj
 0002:00001278       ??_C@_0EC@OFBFCAEJ@?$FLINFO?$FN?3?5WinAccessBridge?3?3getAcc@ 10009278     WinAccessBridge.obj
 0002:000012c0       ??_C@_0JA@MODCAACP@?$FLINFO?$FN?3?5?5?5name?3?5?$CFls?6?5?5?5?5?5?5?5?5?5?5d@ 100092c0     WinAccessBridge.obj
 0002:00001350       ??_C@_0EJ@HLHMECO@?$FLINFO?$FN?3?5WinAccessBridge?3?3getAcc@ 10009350     WinAccessBridge.obj
 0002:000013a0       ??_C@_0EA@MDGJLODH@?$FLINFO?$FN?3?5WinAccessBridge?3?3getAcc@ 100093a0     WinAccessBridge.obj
 0002:000013e0       ??_C@_0EI@IEEMIFOJ@?$FLINFO?$FN?3?5?$CD?$CD?$CD?$CD?$CD?5WinAccessBridge?3?3@ 100093e0     WinAccessBridge.obj
 0002:00001428       ??_C@_0EC@FNKONEFN@?$FLINFO?$FN?3?5?5?5?$CD?$CD?$CD?$CD?$CD?5WinAccessBridge@ 10009428     WinAccessBridge.obj
 0002:00001470       ??_C@_0EA@GPGOILHN@?$FLERROR?$FN?3?5?5?5?$CD?$CD?$CD?$CD?$CD?5WinAccessBridg@ 10009470     WinAccessBridge.obj
 0002:000014b0       ??_C@_0EO@GIFIOBJO@?$FLINFO?$FN?3?5?$CD?$CD?$CD?$CD?$CD?5WinAccessBridge?3?3@ 100094b0     WinAccessBridge.obj
 0002:00001500       ??_C@_0DK@FPHEFKPF@?$FLINFO?$FN?3?5?5?5XXXX?5pkg?9?$DOrTableCellI@ 10009500     WinAccessBridge.obj
 0002:00001540       ??_C@_0EG@CFNEHAJF@?$FLINFO?$FN?3?5?5?5?$CD?$CD?$CD?$CD?$CD?5WinAccessBridge@ 10009540     WinAccessBridge.obj
 0002:00001588       ??_C@_0EE@DMEKGPAL@?$FLERROR?$FN?3?5?5?5?$CD?$CD?$CD?$CD?$CD?5WinAccessBridg@ 10009588     WinAccessBridge.obj
 0002:000015d0       ??_C@_0EJ@GHNOCBA@?$FLINFO?$FN?3?5?$CD?$CD?$CD?$CD?$CD?5WinAccessBridge?3?3@ 100095d0     WinAccessBridge.obj
 0002:00001620       ??_C@_0EH@MMAIEADN@?$FLINFO?$FN?3?5?5?5?$CD?$CD?$CD?$CD?$CD?5WinAccessBridge@ 10009620     WinAccessBridge.obj
 0002:00001668       ??_C@_0EF@IGPDOLOH@?$FLERROR?$FN?3?5?5?5?$CD?$CD?$CD?$CD?$CD?5WinAccessBridg@ 10009668     WinAccessBridge.obj
 0002:000016b0       ??_C@_0EM@KLDOANDG@?$FLINFO?$FN?3?5?$CD?$CD?$CD?$CD?$CD?5WinAccessBridge?3?3@ 100096b0     WinAccessBridge.obj
 0002:00001700       ??_C@_0EK@DJMDCCLK@?$FLINFO?$FN?3?5?5?5?$CD?$CD?$CD?$CD?$CD?5WinAccessBridge@ 10009700     WinAccessBridge.obj
 0002:00001750       ??_C@_0EI@CELDDCKP@?$FLERROR?$FN?3?5?5?5?$CD?$CD?$CD?$CD?$CD?5WinAccessBridg@ 10009750     WinAccessBridge.obj
 0002:00001798       ??_C@_0FC@BPONCABC@?$FLINFO?$FN?3?5?$CD?$CD?$CD?$CD?$CD?5WinAccessBridge?3?3@ 10009798     WinAccessBridge.obj
 0002:000017f0       ??_C@_0EM@JPIPIDPC@?$FLINFO?$FN?3?5?5?5?$CD?$CD?$CD?$CD?$CD?5WinAccessBridge@ 100097f0     WinAccessBridge.obj
 0002:00001840       ??_C@_0EK@IGPCFPOI@?$FLERROR?$FN?3?5?5?5?$CD?$CD?$CD?$CD?$CD?5WinAccessBridg@ 10009840     WinAccessBridge.obj
 0002:00001890       ??_C@_0FF@GEJHIBCC@?$FLINFO?$FN?3?5?$CD?$CD?$CD?$CD?$CD?5WinAccessBridge?3?3@ 10009890     WinAccessBridge.obj
 0002:000018e8       ??_C@_0EP@PJFHLMKB@?$FLINFO?$FN?3?5?5?5?$CD?$CD?$CD?$CD?$CD?5WinAccessBridge@ 100098e8     WinAccessBridge.obj
 0002:00001938       ??_C@_0EN@FJIGOJNI@?$FLERROR?$FN?3?5?5?5?$CD?$CD?$CD?$CD?$CD?5WinAccessBridg@ 10009938     WinAccessBridge.obj
 0002:00001988       ??_C@_0FB@IPIFJJKK@?$FLINFO?$FN?3?5?$CD?$CD?$CD?$CD?$CD?5WinAccessBridge?3?3@ 10009988     WinAccessBridge.obj
 0002:000019e0       ??_C@_0EP@DHAGNOBO@?$FLINFO?$FN?3?5?5?5?$CD?$CD?$CD?$CD?$CD?5WinAccessBridge@ 100099e0     WinAccessBridge.obj
 0002:00001a30       ??_C@_0EN@IFAFODLF@?$FLERROR?$FN?3?5?5?5?$CD?$CD?$CD?$CD?$CD?5WinAccessBridg@ 10009a30     WinAccessBridge.obj
 0002:00001a80       ??_C@_0EK@FCAMCNJB@?$FLINFO?$FN?3?5?$CD?$CD?$CD?$CD?$CD?5WinAccessBridge?3?3@ 10009a80     WinAccessBridge.obj
 0002:00001ad0       ??_C@_0EI@LCHMKLCB@?$FLINFO?$FN?3?5?5?5?$CD?$CD?$CD?$CD?$CD?5WinAccessBridge@ 10009ad0     WinAccessBridge.obj
 0002:00001b18       ??_C@_0EG@PCFFNJPM@?$FLERROR?$FN?3?5?5?5?$CD?$CD?$CD?$CD?$CD?5WinAccessBridg@ 10009b18     WinAccessBridge.obj
 0002:00001b60       ??_C@_0EN@MHFLCDEG@?$FLINFO?$FN?3?5?$CD?$CD?$CD?$CD?$CD?5WinAccessBridge?3?3@ 10009b60     WinAccessBridge.obj
 0002:00001bb0       ??_C@_0EL@HPJEOBAF@?$FLINFO?$FN?3?5?5?5?$CD?$CD?$CD?$CD?$CD?5WinAccessBridge@ 10009bb0     WinAccessBridge.obj
 0002:00001c00       ??_C@_0EJ@EFJNHGOC@?$FLERROR?$FN?3?5?5?5?$CD?$CD?$CD?$CD?$CD?5WinAccessBridg@ 10009c00     WinAccessBridge.obj
 0002:00001c50       ??_C@_0FE@EEAPAHGA@?$FLINFO?$FN?3?5?$CD?$CD?$CD?$CD?$CD?5WinAccessBridge?3?3@ 10009c50     WinAccessBridge.obj
 0002:00001ca8       ??_C@_0FC@IJCKDOEL@?$FLINFO?$FN?3?5?5?5?$CD?$CD?$CD?$CD?$CD?5WinAccessBridge@ 10009ca8     WinAccessBridge.obj
 0002:00001d00       ??_C@_0FA@EEJJLKOB@?$FLERROR?$FN?3?5?5?5?$CD?$CD?$CD?$CD?$CD?5WinAccessBridg@ 10009d00     WinAccessBridge.obj
 0002:00001d50       ??_C@_0EN@IKMAMDCJ@?$FLINFO?$FN?3?5?$CD?$CD?$CD?$CD?$CD?5WinAccessBridge?3?3@ 10009d50     WinAccessBridge.obj
 0002:00001da0       ??_C@_0EL@MCFEFCEP@?$FLINFO?$FN?3?5?5?5?$CD?$CD?$CD?$CD?$CD?5WinAccessBridge@ 10009da0     WinAccessBridge.obj
 0002:00001df0       ??_C@_0EJ@OEGCIAEN@?$FLERROR?$FN?3?5?5?5?$CD?$CD?$CD?$CD?$CD?5WinAccessBridg@ 10009df0     WinAccessBridge.obj
 0002:00001e40       ??_C@_0FB@FBDIFIGA@?$FLERROR?$FN?3?5?$CD?$CD?$CD?$CD?$CD?5WinAccessBridge?3@ 10009e40     WinAccessBridge.obj
 0002:00001e98       ??_C@_0EO@KBJAHINP@?$FLINFO?$FN?3?5?5?5?$CD?$CD?$CD?$CD?$CD?5WinAccessBridge@ 10009e98     WinAccessBridge.obj
 0002:00001ee8       ??_C@_0EM@FBMEIFEO@?$FLERROR?$FN?3?5?5?5?$CD?$CD?$CD?$CD?$CD?5WinAccessBridg@ 10009ee8     WinAccessBridge.obj
 0002:00001f38       ??_C@_0EN@EJPIGDNI@?$FLINFO?$FN?3?5?$CD?$CD?$CD?$CD?$CD?5WinAccessBridge?3?3@ 10009f38     WinAccessBridge.obj
 0002:00001f88       ??_C@_0EB@EHNAMLGG@?$FLINFO?$FN?3?5?5?5?$CD?$CD?$CD?$CD?$CD?5WinAccessBridge@ 10009f88     WinAccessBridge.obj
 0002:00001fcc       ??_C@_0DP@JGIKFGJD@?$FLERROR?$FN?3?5?5?5?$CD?$CD?$CD?$CD?$CD?5WinAccessBridg@ 10009fcc     WinAccessBridge.obj
 0002:00002010       ??_C@_0FA@BNCMMHDE@?$FLINFO?$FN?3?5?$CD?$CD?$CD?$CD?$CD?5WinAccessBridge?3?3@ 1000a010     WinAccessBridge.obj
 0002:00002060       ??_C@_0EE@HJIACDJB@?$FLINFO?$FN?3?5?5?5?$CD?$CD?$CD?$CD?$CD?5WinAccessBridge@ 1000a060     WinAccessBridge.obj
 0002:000020a8       ??_C@_0EC@HJIAKIIH@?$FLERROR?$FN?3?5?5?5?$CD?$CD?$CD?$CD?$CD?5WinAccessBridg@ 1000a0a8     WinAccessBridge.obj
 0002:000020f0       ??_C@_0FF@NCBHFIIB@?$FLINFO?$FN?3?5?$CD?$CD?$CD?$CD?$CD?5WinAccessBridge?3?3@ 1000a0f0     WinAccessBridge.obj
 0002:00002148       ??_C@_0ED@CBAGECAG@?$FLINFO?$FN?3?5?5?5?$CD?$CD?$CD?$CD?$CD?5WinAccessBridge@ 1000a148     WinAccessBridge.obj
 0002:00002190       ??_C@_0EB@NLKCNKIL@?$FLERROR?$FN?3?5?5?5?$CD?$CD?$CD?$CD?$CD?5WinAccessBridg@ 1000a190     WinAccessBridge.obj
 0002:000021d8       ??_C@_0EK@KPCBMLHL@?$FLINFO?$FN?3?5?$CD?$CD?$CD?$CD?$CD?5WinAccessBridge?3?3@ 1000a1d8     WinAccessBridge.obj
 0002:00002228       ??_C@_0ED@KBOKJBJ@?$FLINFO?$FN?3?5?5?5?$CD?$CD?$CD?$CD?$CD?5pkg?9?$DOrAccessibl@ 1000a228     WinAccessBridge.obj
 0002:00002270       ??_C@_0EE@MLCJPFKH@?$FLINFO?$FN?3?5?5?5?$CD?$CD?$CD?$CD?$CD?5WinAccessBridge@ 1000a270     WinAccessBridge.obj
 0002:000022b8       ??_C@_0EC@ONHLHLKJ@?$FLERROR?$FN?3?5?5?5?$CD?$CD?$CD?$CD?$CD?5WinAccessBridg@ 1000a2b8     WinAccessBridge.obj
 0002:00002300       ??_C@_0EI@BEINFODC@?$FLINFO?$FN?3?5?$CD?$CD?$CD?$CD?$CD?5WinAccessBridge?3?3@ 1000a300     WinAccessBridge.obj
 0002:00002348       ??_C@_0CN@CIJKLIHC@?$FLINFO?$FN?3?5?5?5?$CD?$CD?$CD?$CD?$CD?5hypertextInfo?4l@ 1000a348     WinAccessBridge.obj
 0002:00002378       ??_C@_0EC@GJFIBKBJ@?$FLINFO?$FN?3?5?5?5?$CD?$CD?$CD?$CD?$CD?5WinAccessBridge@ 1000a378     WinAccessBridge.obj
 0002:000023c0       ??_C@_0EA@ENIAHHMF@?$FLERROR?$FN?3?5?5?5?$CD?$CD?$CD?$CD?$CD?5WinAccessBridg@ 1000a3c0     WinAccessBridge.obj
 0002:00002400       ??_C@_0EI@MFFNFMHA@?$FLINFO?$FN?3?5WinAccessBridge?3?3activa@ 1000a400     WinAccessBridge.obj
 0002:00002448       ??_C@_0GC@OOPIFCLD@?$FLERROR?$FN?3?5?5WinAccessBridge?3?3acti@ 1000a448     WinAccessBridge.obj
 0002:000024b0       ??_C@_0EJ@KNECEC@?$FLINFO?$FN?3?5?$CD?$CD?$CD?$CD?$CD?5WinAccessBridge?3?3@ 1000a4b0     WinAccessBridge.obj
 0002:000024fc       ??_C@_0CJ@CHHBPBDA@?$FLINFO?$FN?3?5?5?5?$CD?$CD?$CD?$CD?$CD?5hypetext?5link?5c@ 1000a4fc     WinAccessBridge.obj
 0002:00002528       ??_C@_0EG@OFFPNIFM@?$FLINFO?$FN?3?5?5?$CD?$CD?$CD?$CD?$CD?5WinAccessBridge?3@ 1000a528     WinAccessBridge.obj
 0002:00002570       ??_C@_0EF@CJEMCIKC@?$FLERROR?$FN?3?5?5?5?$CD?$CD?$CD?$CD?$CD?5WinAccessBridg@ 1000a570     WinAccessBridge.obj
 0002:000025b8       ??_C@_0EK@KALHBKDC@?$FLINFO?$FN?3?5?$CD?$CD?$CD?$CD?$CD?5WinAccessBridge?3?3@ 1000a5b8     WinAccessBridge.obj
 0002:00002604       ??_C@_0CD@FAKLHPNN@?$FLINFO?$FN?3?5?5?5?$CD?$CD?$CD?$CD?$CD?5pkg?9?$DOrSuccess?5?$DN@ 1000a604     WinAccessBridge.obj
 0002:00002628       ??_C@_0ED@CLMPFLBE@?$FLERROR?$FN?3?5?5?5?$CD?$CD?$CD?$CD?$CD?5WinAccessBridg@ 1000a628     WinAccessBridge.obj
 0002:00002670       ??_C@_0EC@DJBOOIDG@?$FLERROR?$FN?3?5?5?$CD?$CD?$CD?$CD?$CD?5WinAccessBridge@ 1000a670     WinAccessBridge.obj
 0002:000026b8       ??_C@_0EN@IMDNGAME@?$FLINFO?$FN?3?5?$CD?$CD?$CD?$CD?$CD?5WinAccessBridge?3?3@ 1000a6b8     WinAccessBridge.obj
 0002:00002708       ??_C@_0CJ@LGNOCJK@?$FLINFO?$FN?3?5?5?5?$CD?$CD?$CD?$CD?$CD?5hypetext?5link?5i@ 1000a708     WinAccessBridge.obj
 0002:00002738       ??_C@_0EM@KCINDCOI@?$FLINFO?$FN?3?5?5?5?$CD?$CD?$CD?$CD?$CD?5WinAccessBridge@ 1000a738     WinAccessBridge.obj
 0002:00002788       ??_C@_0EI@IEJDJKBK@?$FLERROR?$FN?5?5?$CD?$CD?$CD?$CD?$CD?5WinAccessBridge?3@ 1000a788     WinAccessBridge.obj
 0002:000027d0       ??_C@_0EI@OHHKPFCO@?$FLINFO?$FN?3?5?$CD?$CD?$CD?$CD?$CD?5WinAccessBridge?3?3@ 1000a7d0     WinAccessBridge.obj
 0002:00002818       ??_C@_0EK@CIOPKHEJ@?$FLINFO?$FN?3?5?$CD?$CD?$CD?$CD?$CD?5WinAccessBridge?3?3@ 1000a818     WinAccessBridge.obj
 0002:00002864       ??_C@_0DC@GOKFJHHA@?$FLINFO?$FN?3?5?5?5?$CD?$CD?$CD?$CD?$CD?5keyBindings?4key@ 1000a864     WinAccessBridge.obj
 0002:00002898       ??_C@_0KM@PICKCJIM@?$FLINFO?$FN?3?5?5?5Key?5Binding?5?$CD?5?$CFd?5?5?5?5?5@ 1000a898     WinAccessBridge.obj
 0002:00002948       ??_C@_0EE@LGIDNFJF@?$FLINFO?$FN?3?5?5?5?$CD?$CD?$CD?$CD?$CD?5WinAccessBridge@ 1000a948     WinAccessBridge.obj
 0002:00002990       ??_C@_0EB@PIGLELIJ@?$FLINFO?$FN?3?5?5?5?$CD?$CD?$CD?$CD?$CD?5WinAccessBridge@ 1000a990     WinAccessBridge.obj
 0002:000029d8       ??_C@_0EE@KBJHDGDB@?$FLINFO?$FN?3?5?$CD?$CD?$CD?$CD?$CD?5WinAccessBridge?3?3@ 1000a9d8     WinAccessBridge.obj
 0002:00002a1c       ??_C@_0CG@JNBKIMJN@?$FLINFO?$FN?3?5?5?5?$CD?$CD?$CD?$CD?$CD?5icons?4iconsCoun@ 1000aa1c     WinAccessBridge.obj
 0002:00002a44       ??_C@_0DO@JGGAAEEG@?$FLINFO?$FN?3?5?5?5?$CD?$CD?$CD?$CD?$CD?5WinAccessBridge@ 1000aa44     WinAccessBridge.obj
 0002:00002a84       ??_C@_0DM@PHFGBDGG@?$FLERROR?$FN?3?5?5?5?$CD?$CD?$CD?$CD?$CD?5WinAccessBridg@ 1000aa84     WinAccessBridge.obj
 0002:00002ac0       ??_C@_0EG@EKEEJFO@?$FLINFO?$FN?3?5?$CD?$CD?$CD?$CD?$CD?5WinAccessBridge?3?3@ 1000aac0     WinAccessBridge.obj
 0002:00002b08       ??_C@_0CK@COBILBN@?$FLINFO?$FN?3?5?5?5?$CD?$CD?$CD?$CD?$CD?5actions?4actions@ 1000ab08     WinAccessBridge.obj
 0002:00002b38       ??_C@_0EA@EKDNLNJA@?$FLINFO?$FN?3?5?5?5?$CD?$CD?$CD?$CD?$CD?5WinAccessBridge@ 1000ab38     WinAccessBridge.obj
 0002:00002b78       ??_C@_0DO@HNCGODDL@?$FLERROR?$FN?3?5?5?5?$CD?$CD?$CD?$CD?$CD?5WinAccessBridg@ 1000ab78     WinAccessBridge.obj
 0002:00002bb8       ??_C@_0EH@IJHNMJPE@?$FLINFO?$FN?3?5WinAccessBridge?3?3doAcce@ 1000abb8     WinAccessBridge.obj
 0002:00002c00       ??_C@_0FL@LJNDNJAB@?$FLERROR?$FN?3?5?5?5WinAccessBridge?3?3doA@ 1000ac00     WinAccessBridge.obj
 0002:00002c5c       ??_C@_0DF@LBCGPHPD@?$FLINFO?$FN?3?5WinAccessBridge?3?3setTex@ 1000ac5c     WinAccessBridge.obj
 0002:00002c94       ??_C@_0DJ@BDMKEGCI@?$FLINFO?$FN?3?5WinAccessBridge?3?3getPar@ 1000ac94     WinAccessBridge.obj
 0002:00002cd0       ??_C@_0FE@FILBCBC@?$FLINFO?$FN?3?5?5?5pkg?9?$DOvmID?3?5?$CFX?5?5?5?5?5?5?5?5@ 1000acd0     WinAccessBridge.obj
 0002:00002d24       ??_C@_0CG@EPJKPFNH@?$FLINFO?$FN?3?5?5?5pkg?9?$DOrAccessibleConte@ 1000ad24     WinAccessBridge.obj
 0002:00002d4c       ??_C@_0DJ@LMOBJNAA@?$FLINFO?$FN?3?5WinAccessBridge?3?3getTop@ 1000ad4c     WinAccessBridge.obj
 0002:00002d88       ??_C@_0EB@EGNBJNPN@?$FLINFO?$FN?3?5WinAccessBridge?3?3getPar@ 1000ad88     WinAccessBridge.obj
 0002:00002dcc       ??_C@_0DG@HMAMEAHE@?$FLINFO?$FN?3?5WinAccessBridge?3?3getObj@ 1000adcc     WinAccessBridge.obj
 0002:00002e04       ??_C@_0DL@DIELJEEF@?$FLINFO?$FN?3?5WinAccessBridge?3?3getAct@ 1000ae04     WinAccessBridge.obj
 0002:00002e40       ??_C@_0EA@KKNJCPIF@?$FLINFO?$FN?3?5WinAccessBridge?3?3getVir@ 1000ae40     WinAccessBridge.obj
 0002:00002e80       ??_C@_0EK@LJJEDFEG@?$FLINFO?$FN?3?5?5?5?5?5WinAccessBridge?3?3ge@ 1000ae80     WinAccessBridge.obj
 0002:00002ecc       ??_C@_0DE@NGCOAPLI@?$FLINFO?$FN?3?5WinAccessBridge?3?3reques@ 1000aecc     WinAccessBridge.obj
 0002:00002f00       ??_C@_0EB@LDKGCIL@?$FLINFO?$FN?3?5?5?5?5?5WinAccessBridge?3?3se@ 1000af00     WinAccessBridge.obj
 0002:00002f48       ??_C@_0EK@FKPJFOFL@?$FLINFO?$FN?3?5?5?5?5?5WinAccessBridge?3?3ge@ 1000af48     WinAccessBridge.obj
 0002:00002f94       ??_C@_0DP@PHLAPJAH@?$FLINFO?$FN?3?5WinAccessBridge?3?3getVis@ 1000af94     WinAccessBridge.obj
 0002:00002fd4       ??_C@_0DK@FFJLHNNJ@?$FLINFO?$FN?3?5WinAccessBridge?3?3getVis@ 1000afd4     WinAccessBridge.obj
 0002:00003010       ??_C@_0DM@MCJMMMCP@?$FLINFO?$FN?3?5WinAccessBridge?3?3setCar@ 1000b010     WinAccessBridge.obj
 0002:00003050       ??_C@_0EJ@FBPIKPOJ@?$FLINFO?$FN?3?5WinAccessBridge?3?3getAcc@ 1000b050     WinAccessBridge.obj
 0002:000030a0       ??_C@_0EK@DNDDFNHD@?$FLINFO?$FN?3?5?5?5charCount?3?5?$CFd?5?5?5?5?5?5?5?5@ 1000b0a0     WinAccessBridge.obj
 0002:000030f0       ??_C@_0EG@BGFOEIHE@?$FLINFO?$FN?3?5WinAccessBridge?3?3getAcc@ 1000b0f0     WinAccessBridge.obj
 0002:00003138       ??_C@_0EK@KLCBPNFL@?$FLINFO?$FN?3?5WinAccessBridge?3?3getAcc@ 1000b138     WinAccessBridge.obj
 0002:00003188       ??_C@_0EL@MJHEEFIF@?$FLINFO?$FN?3?5WinAccessBridge?3?3getAcc@ 1000b188     WinAccessBridge.obj
 0002:000031d8       ??_C@_0EF@MMEINAI@?$FLINFO?$FN?3?5WinAccessBridge?3?3getAcc@ 1000b1d8     WinAccessBridge.obj
 0002:00003220       ??_C@_0EA@GJMJEHDC@?$FLINFO?$FN?3?5WinAccessBridge?3?3getCar@ 1000b220     WinAccessBridge.obj
 0002:00003260       ??_C@_0EJ@BCHIKCEF@?$FLINFO?$FN?3?5WinAccessBridge?3?3getAcc@ 1000b260     WinAccessBridge.obj
 0002:000032b0       ??_C@_0EI@LCFAOBKP@?$FLINFO?$FN?3?5WinAccessBridge?3?3getAcc@ 1000b2b0     WinAccessBridge.obj
 0002:000032f8       ??_C@_0DM@NFGOCJPM@?$FLINFO?$FN?3?5WinAccessBridge?3?3addJav@ 1000b2f8     WinAccessBridge.obj
 0002:00003334       ??_C@_0DP@PIGNLFHB@?$FLINFO?$FN?3?5?5?5?9?$DOpkgType?5?$DN?5?$CFX?0?5event@ 1000b334     WinAccessBridge.obj
 0002:00003378       ??_C@_0EC@OKCIJGM@?$FLINFO?$FN?3?5in?5WinAccessBridge?3?3rem@ 1000b378     WinAccessBridge.obj
 0002:000033c0       ??_C@_0EI@HMKIAPB@?$FLINFO?$FN?3?5in?5WinAccessBridge?3?3add@ 1000b3c0     WinAccessBridge.obj
 0002:00003408       ??_C@_0DP@KFDABLNL@?$FLINFO?$FN?3?5?5?5?9?$DOpkgType?5?$DN?5?$CFX?0?5event@ 1000b408     WinAccessBridge.obj
 0002:00003448       ??_C@_0EL@BFCCGHFN@?$FLINFO?$FN?3?5in?5WinAccessBridge?3?3rem@ 1000b448     WinAccessBridge.obj
 0002:00003498       ??_7type_info@@6B@         1000b498     MSVCRT:std_type_info_static.obj
 0002:0000349c       __pRawDllMain              1000b49c     MSVCRT:dll_dllmain.obj
 0002:0000349c       __pDefaultRawDllMain       1000b49c     MSVCRT:dll_dllmain.obj
 0002:000034ac       ??_7bad_array_new_length@std@@6B@ 1000b4ac     MSVCRT:throw_bad_alloc.obj
 0002:000034b4       ??_C@_0BF@KINCDENJ@bad?5array?5new?5length@ 1000b4b4     MSVCRT:throw_bad_alloc.obj
 0002:00003540       __load_config_used         1000b540     MSVCRT:loadcfg.obj
 0002:000035f8       ??_R4exception@std@@6B@    1000b5f8     AccessBridgeMessageQueue.obj
 0002:0000360c       ??_R3exception@std@@8      1000b60c     AccessBridgeMessageQueue.obj
 0002:0000361c       ??_R2exception@std@@8      1000b61c     AccessBridgeMessageQueue.obj
 0002:00003624       ??_R1A@?0A@EA@exception@std@@8 1000b624     AccessBridgeMessageQueue.obj
 0002:00003640       ??_R4bad_alloc@std@@6B@    1000b640     AccessBridgeMessageQueue.obj
 0002:00003654       ??_R3bad_alloc@std@@8      1000b654     AccessBridgeMessageQueue.obj
 0002:00003664       ??_R2bad_alloc@std@@8      1000b664     AccessBridgeMessageQueue.obj
 0002:00003670       ??_R1A@?0A@EA@bad_alloc@std@@8 1000b670     AccessBridgeMessageQueue.obj
 0002:0000368c       ??_R4type_info@@6B@        1000b68c     MSVCRT:std_type_info_static.obj
 0002:000036a0       ??_R3type_info@@8          1000b6a0     MSVCRT:std_type_info_static.obj
 0002:000036b0       ??_R2type_info@@8          1000b6b0     MSVCRT:std_type_info_static.obj
 0002:000036b8       ??_R1A@?0A@EA@type_info@@8 1000b6b8     MSVCRT:std_type_info_static.obj
 0002:000036d4       ??_R4bad_array_new_length@std@@6B@ 1000b6d4     MSVCRT:throw_bad_alloc.obj
 0002:000036e8       ??_R3bad_array_new_length@std@@8 1000b6e8     MSVCRT:throw_bad_alloc.obj
 0002:000036f8       ??_R2bad_array_new_length@std@@8 1000b6f8     MSVCRT:throw_bad_alloc.obj
 0002:00003708       ??_R1A@?0A@EA@bad_array_new_length@std@@8 1000b708     MSVCRT:throw_bad_alloc.obj
 0002:00003724       ___safe_se_handler_table   1000b724     <linker-defined>
 0002:000039e0       ___rtc_iaa                 1000b9e0     MSVCRT:initsect.obj
 0002:000039e4       ___rtc_izz                 1000b9e4     MSVCRT:initsect.obj
 0002:000039e8       ___rtc_taa                 1000b9e8     MSVCRT:initsect.obj
 0002:000039ec       ___rtc_tzz                 1000b9ec     MSVCRT:initsect.obj
 0002:000039f0       __CT??_R0?AVbad_alloc@std@@@8??0bad_alloc@std@@QAE@ABV01@@Z12 1000b9f0     AccessBridgeMessageQueue.obj
 0002:00003a0c       __CT??_R0?AVexception@std@@@8??0exception@std@@QAE@ABV01@@Z12 1000ba0c     AccessBridgeMessageQueue.obj
 0002:00003a28       __TI2?AVbad_alloc@std@@    1000ba28     AccessBridgeMessageQueue.obj
 0002:00003a38       __CTA2?AVbad_alloc@std@@   1000ba38     AccessBridgeMessageQueue.obj
 0002:00003aac       __TI3?AVbad_array_new_length@std@@ 1000baac     MSVCRT:throw_bad_alloc.obj
 0002:00003abc       __CTA3?AVbad_array_new_length@std@@ 1000babc     MSVCRT:throw_bad_alloc.obj
 0002:00003acc       __CT??_R0?AVbad_array_new_length@std@@@8??0bad_array_new_length@std@@QAE@ABV01@@Z12 1000bacc     MSVCRT:throw_bad_alloc.obj
 0002:00004954       __IMPORT_DESCRIPTOR_KERNEL32 1000c954     kernel32:KERNEL32.dll
 0002:00004968       __IMPORT_DESCRIPTOR_USER32 1000c968     user32:USER32.dll
 0002:0000497c       __IMPORT_DESCRIPTOR_VCRUNTIME140 1000c97c     vcruntime:VCRUNTIME140.dll
 0002:00004990       __IMPORT_DESCRIPTOR_api-ms-win-crt-string-l1-1-0 1000c990     ucrt:api-ms-win-crt-string-l1-1-0.dll
 0002:000049a4       __IMPORT_DESCRIPTOR_api-ms-win-crt-stdio-l1-1-0 1000c9a4     ucrt:api-ms-win-crt-stdio-l1-1-0.dll
 0002:000049b8       __IMPORT_DESCRIPTOR_api-ms-win-crt-environment-l1-1-0 1000c9b8     ucrt:api-ms-win-crt-environment-l1-1-0.dll
 0002:000049cc       __IMPORT_DESCRIPTOR_api-ms-win-crt-heap-l1-1-0 1000c9cc     ucrt:api-ms-win-crt-heap-l1-1-0.dll
 0002:000049e0       __IMPORT_DESCRIPTOR_api-ms-win-crt-runtime-l1-1-0 1000c9e0     ucrt:api-ms-win-crt-runtime-l1-1-0.dll
 0002:000049f4       __NULL_IMPORT_DESCRIPTOR   1000c9f4     kernel32:KERNEL32.dll
 0003:00000000       ___security_cookie_complement 1000e000     MSVCRT:gs_cookie.obj
 0003:00000004       ___security_cookie         1000e004     MSVCRT:gs_cookie.obj
 0003:00000010       ___scrt_native_dllmain_reason 1000e010     MSVCRT:utility.obj
 0003:00000020       ___isa_enabled             1000e020     MSVCRT:cpu_disp.obj
 0003:00000024       ___scrt_ucrt_dll_is_in_use 1000e024     MSVCRT:ucrt_stubs.obj
 0003:00000028       ??_R0?AVbad_alloc@std@@@8  1000e028     AccessBridgeMessageQueue.obj
 0003:00000044       ??_R0?AVexception@std@@@8  1000e044     AccessBridgeMessageQueue.obj
 0003:00000060       ??_R0?AVtype_info@@@8      1000e060     MSVCRT:std_type_info_static.obj
 0003:00000078       ??_R0?AVbad_array_new_length@std@@@8 1000e078     MSVCRT:throw_bad_alloc.obj
 0003:000000a0       ?_OptionsStorage@?1??__local_stdio_printf_options@@9@4_KA 1000e0a0     AccessBridgeDebug.obj
 0003:000000ac       ?theFromJavaHelloMsgID@@3IA 1000e0ac     AccessBridgeMessages.obj
 0003:000000b0       ?theFromWindowsHelloMsgID@@3IA 1000e0b0     AccessBridgeMessages.obj
 0003:000000b4       ?sendMemoryIPCLock@@3U_RTL_CRITICAL_SECTION@@A 1000e0b4     WinAccessBridge.obj
 0003:000000cc       ?newJVMs@@3PAPADA          1000e0cc     WinAccessBridge.obj
 0003:000000d0       ?theWindowsAccessBridge@@3PAVWinAccessBridge@@A 1000e0d0     WinAccessBridge.obj
 0003:000000d4       ?theDialogWindow@@3PAUHWND__@@A 1000e0d4     WinAccessBridge.obj
 0003:000000d8       ?isVMInstanceChainInUse@@3_NA 1000e0d8     WinAccessBridge.obj
 0003:00000400       ?__type_info_root_node@@3U__type_info_node@@A 1000e400     MSVCRT:tncleanup.obj
 0003:00000408       ?_OptionsStorage@?1??__local_stdio_scanf_options@@9@4_KA 1000e408     MSVCRT:default_local_stdio_options.obj
 0003:00000410       ___scrt_current_native_startup_state 1000e410     MSVCRT:utility.obj
 0003:00000414       ___scrt_native_startup_lock 1000e414     MSVCRT:utility.obj
 0003:00000434       ___scrt_debugger_hook_flag 1000e434     MSVCRT:utility_desktop.obj
 0003:00000438       ___isa_available           1000e438     MSVCRT:cpu_disp.obj
 0003:0000043c       ___favor                   1000e43c     MSVCRT:cpu_disp.obj
 0003:00000440       ___dyn_tls_init_callback   1000e440     <common>

 entry point at        0001:000061fd

 Static symbols

 0000:fffef000       .debug$S                   10000000     windowsaccessbridge-32.exp
 0000:fffef000       .debug$S                   10000000     vcruntime:VCRUNTIME140.dll
 0000:fffef000       .debug$S                   10000000     vcruntime:VCRUNTIME140.dll
 0000:fffef000       .debug$S                   10000000     vcruntime:VCRUNTIME140.dll
 0000:fffef000       .debug$S                   10000000     vcruntime:VCRUNTIME140.dll
 0000:fffef000       .debug$S                   10000000     vcruntime:VCRUNTIME140.dll
 0000:fffef000       .debug$S                   10000000     vcruntime:VCRUNTIME140.dll
 0000:fffef000       .debug$S                   10000000     vcruntime:VCRUNTIME140.dll
 0000:fffef000       .debug$S                   10000000     vcruntime:VCRUNTIME140.dll
 0000:fffef000       .debug$S                   10000000     vcruntime:VCRUNTIME140.dll
 0000:fffef000       .debug$S                   10000000     ucrt:api-ms-win-crt-environment-l1-1-0.dll
 0000:fffef000       .debug$S                   10000000     ucrt:api-ms-win-crt-heap-l1-1-0.dll
 0000:fffef000       .debug$S                   10000000     ucrt:api-ms-win-crt-heap-l1-1-0.dll
 0000:fffef000       .debug$S                   10000000     ucrt:api-ms-win-crt-heap-l1-1-0.dll
 0000:fffef000       .debug$S                   10000000     ucrt:api-ms-win-crt-runtime-l1-1-0.dll
 0000:fffef000       .debug$S                   10000000     ucrt:api-ms-win-crt-runtime-l1-1-0.dll
 0000:fffef000       .debug$S                   10000000     ucrt:api-ms-win-crt-runtime-l1-1-0.dll
 0000:fffef000       .debug$S                   10000000     ucrt:api-ms-win-crt-runtime-l1-1-0.dll
 0000:fffef000       .debug$S                   10000000     ucrt:api-ms-win-crt-runtime-l1-1-0.dll
 0000:fffef000       .debug$S                   10000000     ucrt:api-ms-win-crt-runtime-l1-1-0.dll
 0000:fffef000       .debug$S                   10000000     ucrt:api-ms-win-crt-runtime-l1-1-0.dll
 0000:fffef000       .debug$S                   10000000     ucrt:api-ms-win-crt-runtime-l1-1-0.dll
 0000:fffef000       .debug$S                   10000000     ucrt:api-ms-win-crt-runtime-l1-1-0.dll
 0000:fffef000       .debug$S                   10000000     ucrt:api-ms-win-crt-runtime-l1-1-0.dll
 0000:fffef000       .debug$S                   10000000     ucrt:api-ms-win-crt-runtime-l1-1-0.dll
 0000:fffef000       .debug$S                   10000000     ucrt:api-ms-win-crt-runtime-l1-1-0.dll
 0000:fffef000       .debug$S                   10000000     ucrt:api-ms-win-crt-stdio-l1-1-0.dll
 0000:fffef000       .debug$S                   10000000     ucrt:api-ms-win-crt-stdio-l1-1-0.dll
 0000:fffef000       .debug$S                   10000000     ucrt:api-ms-win-crt-stdio-l1-1-0.dll
 0000:fffef000       .debug$S                   10000000     ucrt:api-ms-win-crt-stdio-l1-1-0.dll
 0000:fffef000       .debug$S                   10000000     ucrt:api-ms-win-crt-stdio-l1-1-0.dll
 0000:fffef000       .debug$S                   10000000     ucrt:api-ms-win-crt-stdio-l1-1-0.dll
 0000:fffef000       .debug$S                   10000000     ucrt:api-ms-win-crt-string-l1-1-0.dll
 0000:fffef000       .debug$S                   10000000     ucrt:api-ms-win-crt-string-l1-1-0.dll
 0000:fffef000       .debug$S                   10000000     ucrt:api-ms-win-crt-string-l1-1-0.dll
 0000:fffef000       .debug$S                   10000000     ucrt:api-ms-win-crt-string-l1-1-0.dll
 0000:fffef000       .debug$S                   10000000     ucrt:api-ms-win-crt-string-l1-1-0.dll
 0000:fffef000       .debug$S                   10000000     ucrt:api-ms-win-crt-string-l1-1-0.dll
 0000:fffef000       .debug$S                   10000000     kernel32:KERNEL32.dll
 0000:fffef000       .debug$S                   10000000     kernel32:KERNEL32.dll
 0000:fffef000       .debug$S                   10000000     kernel32:KERNEL32.dll
 0000:fffef000       .debug$S                   10000000     kernel32:KERNEL32.dll
 0000:fffef000       .debug$S                   10000000     kernel32:KERNEL32.dll
 0000:fffef000       .debug$S                   10000000     kernel32:KERNEL32.dll
 0000:fffef000       .debug$S                   10000000     kernel32:KERNEL32.dll
 0000:fffef000       .debug$S                   10000000     kernel32:KERNEL32.dll
 0000:fffef000       .debug$S                   10000000     kernel32:KERNEL32.dll
 0000:fffef000       .debug$S                   10000000     kernel32:KERNEL32.dll
 0000:fffef000       .debug$S                   10000000     kernel32:KERNEL32.dll
 0000:fffef000       .debug$S                   10000000     kernel32:KERNEL32.dll
 0000:fffef000       .debug$S                   10000000     kernel32:KERNEL32.dll
 0000:fffef000       .debug$S                   10000000     kernel32:KERNEL32.dll
 0000:fffef000       .debug$S                   10000000     kernel32:KERNEL32.dll
 0000:fffef000       .debug$S                   10000000     kernel32:KERNEL32.dll
 0000:fffef000       .debug$S                   10000000     kernel32:KERNEL32.dll
 0000:fffef000       .debug$S                   10000000     kernel32:KERNEL32.dll
 0000:fffef000       .debug$S                   10000000     kernel32:KERNEL32.dll
 0000:fffef000       .debug$S                   10000000     kernel32:KERNEL32.dll
 0000:fffef000       .debug$S                   10000000     kernel32:KERNEL32.dll
 0000:fffef000       .debug$S                   10000000     kernel32:KERNEL32.dll
 0000:fffef000       .debug$S                   10000000     kernel32:KERNEL32.dll
 0000:fffef000       .debug$S                   10000000     kernel32:KERNEL32.dll
 0000:fffef000       .debug$S                   10000000     user32:USER32.dll
 0000:fffef000       .debug$S                   10000000     user32:USER32.dll
 0000:fffef000       .debug$S                   10000000     user32:USER32.dll
 0000:fffef000       .debug$S                   10000000     user32:USER32.dll
 0000:fffef000       .debug$S                   10000000     user32:USER32.dll
 0000:fffef000       .debug$S                   10000000     user32:USER32.dll
 0000:fffef000       .debug$S                   10000000     user32:USER32.dll
 0000:fffef000       .debug$S                   10000000     user32:USER32.dll
 0000:fffef000       .debug$S                   10000000     user32:USER32.dll
 0000:fffef000       .debug$S                   10000000     user32:USER32.dll
 0000:fffef000       .debug$S                   10000000     user32:USER32.dll
 0000:fffef000       .debug$S                   10000000     user32:USER32.dll
 0000:fffef000       .debug$S                   10000000     user32:USER32.dll
 0001:00005db0       $$000000                   10006db0     MSVCRT:ulldiv.obj
 0001:00005e90       $$000000                   10006e90     MSVCRT:chkstk.obj
 0001:00005ebd       ?dllmain_crt_dispatch@@YGHQAUHINSTANCE__@@KQAX@Z 10006ebd f   MSVCRT:dll_dllmain.obj
 0001:00005f10       ?dllmain_crt_process_attach@@YAHQAUHINSTANCE__@@QAX@Z 10006f10 f   MSVCRT:dll_dllmain.obj
 0001:00006017       ?dllmain_crt_process_detach@@YAH_N@Z 10007017 f   MSVCRT:dll_dllmain.obj
 0001:000060c7       ?dllmain_dispatch@@YAHQAUHINSTANCE__@@KQAX@Z 100070c7 f   MSVCRT:dll_dllmain.obj
 0001:000061d2       ?dllmain_raw@@YGHQAUHINSTANCE__@@KQAX@Z 100071d2 f   MSVCRT:dll_dllmain.obj
 0001:000063e0       ___get_entropy             100073e0 f   MSVCRT:gs_support.obj
 0001:000064b3       ?find_pe_section@@YAPAU_IMAGE_SECTION_HEADER@@QAEI@Z 100074b3 f   MSVCRT:utility.obj
 0001:00006910       $$000000                   10007910     MSVCRT:sehprolg4.obj
 0002:000034a0       _GS_ExceptionPointers      1000b4a0     MSVCRT:gs_report.obj
 0002:00003a48       __sehtable$?dllmain_crt_process_attach@@YAHQAUHINSTANCE__@@QAX@Z 1000ba48     MSVCRT:dll_dllmain.obj
 0002:00003a68       __sehtable$?dllmain_crt_process_detach@@YAH_N@Z 1000ba68     MSVCRT:dll_dllmain.obj
 0002:00003a90       __sehtable$?dllmain_dispatch@@YAHQAUHINSTANCE__@@KQAX@Z 1000ba90     MSVCRT:dll_dllmain.obj
 0002:00003ae8       __sehtable$___scrt_is_nonwritable_in_current_image 1000bae8     MSVCRT:utility.obj
 0002:00003b10       .edata                     1000bb10     windowsaccessbridge-32.exp
 0002:00003b38       rgpv                       1000bb38     windowsaccessbridge-32.exp
 0002:00003ccc       rgszName                   1000bccc     windowsaccessbridge-32.exp
 0002:00003e60       rgwOrd                     1000be60     windowsaccessbridge-32.exp
 0002:00003f2a       szName                     1000bf2a     windowsaccessbridge-32.exp
 0002:00003f45       $N00001                    1000bf45     windowsaccessbridge-32.exp
 0002:00003f67       $N00002                    1000bf67     windowsaccessbridge-32.exp
 0002:00003f80       $N00003                    1000bf80     windowsaccessbridge-32.exp
 0002:00003fa5       $N00004                    1000bfa5     windowsaccessbridge-32.exp
 0002:00003fc1       $N00005                    1000bfc1     windowsaccessbridge-32.exp
 0002:00003fcd       $N00006                    1000bfcd     windowsaccessbridge-32.exp
 0002:00003fe9       $N00007                    1000bfe9     windowsaccessbridge-32.exp
 0002:0000400b       $N00008                    1000c00b     windowsaccessbridge-32.exp
 0002:0000402f       $N00009                    1000c02f     windowsaccessbridge-32.exp
 0002:00004043       $N00010                    1000c043     windowsaccessbridge-32.exp
 0002:00004058       $N00011                    1000c058     windowsaccessbridge-32.exp
 0002:00004076       $N00012                    1000c076     windowsaccessbridge-32.exp
 0002:0000408d       $N00013                    1000c08d     windowsaccessbridge-32.exp
 0002:000040aa       $N00014                    1000c0aa     windowsaccessbridge-32.exp
 0002:000040c3       $N00015                    1000c0c3     windowsaccessbridge-32.exp
 0002:000040e1       $N00016                    1000c0e1     windowsaccessbridge-32.exp
 0002:000040f8       $N00017                    1000c0f8     windowsaccessbridge-32.exp
 0002:00004114       $N00018                    1000c114     windowsaccessbridge-32.exp
 0002:0000412b       $N00019                    1000c12b     windowsaccessbridge-32.exp
 0002:00004145       $N00020                    1000c145     windowsaccessbridge-32.exp
 0002:00004165       $N00021                    1000c165     windowsaccessbridge-32.exp
 0002:00004178       $N00022                    1000c178     windowsaccessbridge-32.exp
 0002:00004191       $N00023                    1000c191     windowsaccessbridge-32.exp
 0002:000041b0       $N00024                    1000c1b0     windowsaccessbridge-32.exp
 0002:000041c9       $N00025                    1000c1c9     windowsaccessbridge-32.exp
 0002:000041f0       $N00026                    1000c1f0     windowsaccessbridge-32.exp
 0002:00004212       $N00027                    1000c212     windowsaccessbridge-32.exp
 0002:0000422d       $N00028                    1000c22d     windowsaccessbridge-32.exp
 0002:00004246       $N00029                    1000c246     windowsaccessbridge-32.exp
 0002:0000426a       $N00030                    1000c26a     windowsaccessbridge-32.exp
 0002:00004289       $N00031                    1000c289     windowsaccessbridge-32.exp
 0002:000042b0       $N00032                    1000c2b0     windowsaccessbridge-32.exp
 0002:000042d3       $N00033                    1000c2d3     windowsaccessbridge-32.exp
 0002:000042eb       $N00034                    1000c2eb     windowsaccessbridge-32.exp
 0002:00004302       $N00035                    1000c302     windowsaccessbridge-32.exp
 0002:00004318       $N00036                    1000c318     windowsaccessbridge-32.exp
 0002:00004339       $N00037                    1000c339     windowsaccessbridge-32.exp
 0002:00004355       $N00038                    1000c355     windowsaccessbridge-32.exp
 0002:00004379       $N00039                    1000c379     windowsaccessbridge-32.exp
 0002:00004399       $N00040                    1000c399     windowsaccessbridge-32.exp
 0002:000043b5       $N00041                    1000c3b5     windowsaccessbridge-32.exp
 0002:000043cb       $N00042                    1000c3cb     windowsaccessbridge-32.exp
 0002:000043e2       $N00043                    1000c3e2     windowsaccessbridge-32.exp
 0002:000043fe       $N00044                    1000c3fe     windowsaccessbridge-32.exp
 0002:00004415       $N00045                    1000c415     windowsaccessbridge-32.exp
 0002:0000442b       $N00046                    1000c42b     windowsaccessbridge-32.exp
 0002:0000444a       $N00047                    1000c44a     windowsaccessbridge-32.exp
 0002:0000445e       $N00048                    1000c45e     windowsaccessbridge-32.exp
 0002:0000446f       $N00049                    1000c46f     windowsaccessbridge-32.exp
 0002:00004494       $N00050                    1000c494     windowsaccessbridge-32.exp
 0002:000044a5       $N00051                    1000c4a5     windowsaccessbridge-32.exp
 0002:000044c2       $N00052                    1000c4c2     windowsaccessbridge-32.exp
 0002:000044e7       $N00053                    1000c4e7     windowsaccessbridge-32.exp
 0002:0000450c       $N00054                    1000c50c     windowsaccessbridge-32.exp
 0002:0000451b       $N00055                    1000c51b     windowsaccessbridge-32.exp
 0002:0000452d       $N00056                    1000c52d     windowsaccessbridge-32.exp
 0002:00004547       $N00057                    1000c547     windowsaccessbridge-32.exp
 0002:00004560       $N00058                    1000c560     windowsaccessbridge-32.exp
 0002:00004572       $N00059                    1000c572     windowsaccessbridge-32.exp
 0002:00004581       $N00060                    1000c581     windowsaccessbridge-32.exp
 0002:0000459a       $N00061                    1000c59a     windowsaccessbridge-32.exp
 0002:000045ad       $N00062                    1000c5ad     windowsaccessbridge-32.exp
 0002:000045c5       $N00063                    1000c5c5     windowsaccessbridge-32.exp
 0002:000045ea       $N00064                    1000c5ea     windowsaccessbridge-32.exp
 0002:0000460a       $N00065                    1000c60a     windowsaccessbridge-32.exp
 0002:00004627       $N00066                    1000c627     windowsaccessbridge-32.exp
 0002:00004634       $N00067                    1000c634     windowsaccessbridge-32.exp
 0002:00004641       $N00068                    1000c641     windowsaccessbridge-32.exp
 0002:00004653       $N00069                    1000c653     windowsaccessbridge-32.exp
 0002:00004678       $N00070                    1000c678     windowsaccessbridge-32.exp
 0002:00004685       $N00071                    1000c685     windowsaccessbridge-32.exp
 0002:000046ad       $N00072                    1000c6ad     windowsaccessbridge-32.exp
 0002:000046bd       $N00073                    1000c6bd     windowsaccessbridge-32.exp
 0002:000046ce       $N00074                    1000c6ce     windowsaccessbridge-32.exp
 0002:000046df       $N00075                    1000c6df     windowsaccessbridge-32.exp
 0002:000046f0       $N00076                    1000c6f0     windowsaccessbridge-32.exp
 0002:000046ff       $N00077                    1000c6ff     windowsaccessbridge-32.exp
 0002:00004711       $N00078                    1000c711     windowsaccessbridge-32.exp
 0002:00004723       $N00079                    1000c723     windowsaccessbridge-32.exp
 0002:00004737       $N00080                    1000c737     windowsaccessbridge-32.exp
 0002:00004749       $N00081                    1000c749     windowsaccessbridge-32.exp
 0002:0000475b       $N00082                    1000c75b     windowsaccessbridge-32.exp
 0002:0000476d       $N00083                    1000c76d     windowsaccessbridge-32.exp
 0002:0000477e       $N00084                    1000c77e     windowsaccessbridge-32.exp
 0002:00004790       $N00085                    1000c790     windowsaccessbridge-32.exp
 0002:000047a3       $N00086                    1000c7a3     windowsaccessbridge-32.exp
 0002:000047ba       $N00087                    1000c7ba     windowsaccessbridge-32.exp
 0002:000047dc       $N00088                    1000c7dc     windowsaccessbridge-32.exp
 0002:000047fc       $N00089                    1000c7fc     windowsaccessbridge-32.exp
 0002:00004820       $N00090                    1000c820     windowsaccessbridge-32.exp
 0002:00004839       $N00091                    1000c839     windowsaccessbridge-32.exp
 0002:0000484d       $N00092                    1000c84d     windowsaccessbridge-32.exp
 0002:00004866       $N00093                    1000c866     windowsaccessbridge-32.exp
 0002:00004885       $N00094                    1000c885     windowsaccessbridge-32.exp
 0002:0000489d       $N00095                    1000c89d     windowsaccessbridge-32.exp
 0002:000048ba       $N00096                    1000c8ba     windowsaccessbridge-32.exp
 0002:000048d3       $N00097                    1000c8d3     windowsaccessbridge-32.exp
 0002:000048f1       $N00098                    1000c8f1     windowsaccessbridge-32.exp
 0002:00004909       $N00099                    1000c909     windowsaccessbridge-32.exp
 0002:00004922       $N00100                    1000c922     windowsaccessbridge-32.exp
 0002:00004941       $N00101                    1000c941     windowsaccessbridge-32.exp
 0002:00004bcc       .idata$6                   1000cbcc     kernel32:KERNEL32.dll
 0002:00004c88       .idata$6                   1000cc88     user32:USER32.dll
 0002:00004d2a       .idata$6                   1000cd2a     vcruntime:VCRUNTIME140.dll
 0002:00004e94       .idata$6                   1000ce94     ucrt:api-ms-win-crt-string-l1-1-0.dll
 0002:00004eb6       .idata$6                   1000ceb6     ucrt:api-ms-win-crt-stdio-l1-1-0.dll
 0002:00004ed6       .idata$6                   1000ced6     ucrt:api-ms-win-crt-environment-l1-1-0.dll
 0002:00004efc       .idata$6                   1000cefc     ucrt:api-ms-win-crt-heap-l1-1-0.dll
 0002:00004f1c       .idata$6                   1000cf1c     ucrt:api-ms-win-crt-runtime-l1-1-0.dll
 0003:000000a8       _logFP                     1000e0a8     AccessBridgeDebug.obj
 0003:000000dc       ?__proc_attached@@3HA      1000e0dc     MSVCRT:dll_dllmain.obj
 0003:000000e0       _GS_ExceptionRecord        1000e0e0     MSVCRT:gs_report.obj
 0003:00000130       _GS_ContextRecord          1000e130     MSVCRT:gs_report.obj
 0003:00000418       ?is_initialized_as_dll@@3_NA 1000e418     MSVCRT:utility.obj
 0003:00000419       ?module_local_atexit_table_initialized@@3_NA 1000e419     MSVCRT:utility.obj
 0003:0000041c       ?module_local_atexit_table@@3U_onexit_table_t@@A 1000e41c     MSVCRT:utility.obj
 0003:00000428       ?module_local_at_quick_exit_table@@3U_onexit_table_t@@A 1000e428     MSVCRT:utility.obj
 0004:00000120       $R000000                   1000f120     windowsaccessbridge-32.dll.res
 0004:000004c0       $R0003A0                   1000f4c0     windowsaccessbridge-32.dll.res
 0004:000006d8       $R0005B8                   1000f6d8     windowsaccessbridge-32.dll.res
